:100000000C9418080C9433080C9433080C9433089F
:100010000C9433080C9433080C9433080C94330874
:100020000C9433080C9433080C9433080C94330864
:100030000C9433080C9433080C9433080C94330854
:100040000C9433080C9433080C94FD120C94330870
:100050000C94010B0C9433080C94C80A0C943308CC
:100060000C94061B0C9433080C9433080C9433083E
:100070000C94A50F0C9433080C9433080D0A0D0A48
:1000800048573A20466F6C6C6F772D4D65000D0A0E
:10009000466F6C6C6F77204D650A0D536F667477F1
:1000A0006172653A5625642E2564256320000D0A89
:1000B0002D2D2D2D2D2D2D2D2D2D2D2D2D2D2D2D70
:1000C0002D2D2D2D2D2D2D2D2D2D2D2D2D2D000DAD
:1000D0000A00416E616C6F675F436830202020200A
:1000E0002020416E616C6F675F43683120202020C3
:1000F0002020416E616C6F675F43683220202020B2
:100100002020416E616C6F675F43683320202020A0
:100110002020416E616C6F675F436834202020208F
:100120002020416E616C6F675F436835202020207E
:100130002020416E616C6F675F436836202020206D
:100140002020416E616C6F675F436837202020205C
:1001500020205542617420202020202020202020B3
:10016000202053797353746174652020202020204F
:100170002020446562756731302020202020202017
:100180002020446562756731312020202020202006
:1001900020204465627567313220202020202020F5
:1001A00020204465627567313320202020202020E4
:1001B00020204465627567313420202020202020D3
:1001C00020204465627567313520202020202020C2
:1001D00020205A656C6C656E7A61686C2020202046
:1001E0002020506F7765724F6E2020202020202025
:1001F000202044656275673138202020202020208F
:10020000202044656275673139202020202020207D
:100210002020446562756732302020202020202075
:100220002020446562756732312020202020202064
:100230002020446562756732322020202020202053
:100240002020446562756732332020202020202042
:100250002020446562756732342020202020202031
:100260002020446562756732352020202020202020
:10027000202044656275673236202020202020200F
:1002800020204465627567323720202020202020FE
:1002900020204465627567323820202020202020ED
:1002A00020204465627567323920202020202020DC
:1002B00020204465627567333020202020202020D4
:1002C00020204465627567333120202020202020C3
:1002D00020200D0A20554152543020696E69742E39
:1002E0002E2E6F6B000D0A20554152543120696E3D
:1002F00069742E2E2E006F6B005B25695D005B25F7
:10030000695D002B20466F6C6C6F77204D65202B4C
:100310000048573A20466F6C6C6F772D4D6500533F
:10032000573A2025642E25642563002020202020B4
:100330002020202020004E6F2047505320646174FD
:1003400061004C6F6E3A20202020202020202020A9
:10035000202020202020004C61743A2020202020E2
:10036000202020202020202020202000416C743AD2
:10037000202020202020202020202020202020207D
:1003800000536174733A25303264204669783A4EDE
:100390006F6E6500536174733A253032642046698C
:1003A000783A3244202000536174733A2530326425
:1003B000204669783A3344202000536174733A250B
:1003C000303264204669783A3F3F2020004C6F6EFF
:1003D0003A20256325642E252E3364252E33642090
:1003E000646567004C61743A20256325642E252ED0
:1003F0003364252E33642064656700416C743A20B1
:100400002563253034642E252E303364206D004E54
:100410006F204750532064617461005370656564B8
:10042000204E3A20202020202020202020202000A4
:10043000537065656420453A20202020202020202C
:100440002020202000537065656420543A2020202D
:1004500020202020202020202000536174733A2582
:10046000303264204669783A4E6F6E65005361748D
:10047000733A25303264204669783A3244202000AD
:10048000536174733A25303264204669783A3344B4
:10049000202000536174733A253032642046697815
:1004A0003A3F3F2020005370656564204E3A202576
:1004B0002B346420636D2F73005370656564204591
:1004C0003A20252B346420636D2F730053706565CB
:1004D0006420543A20252B346420636D2F73004729
:1004E0005053205554432054696D6500202020202E
:1004F00020202020202020202020202020202020FC
:100500000020204E6F2074696D6520646174612144
:1005100020202020200020202020202020202020FB
:1005200020202020202020202020002020202020EB
:1005300020202020202020202020202020202000DB
:10054000446174653A20253032692F253032692F95
:10055000253034690054696D653A20253032693A96
:10056000253032693A253032692E25303369000D45
:100570000A2055425820696E69742E2E2E006F6B2A
:10058000000D0A2041444320696E69742E2E2E000E
:100590006F6B000D0A20425554544F4E20696E690E
:1005A000742E2E2E006F6B0000002110422063304D
:1005B0008440A550C660E770088129914AA16BB1BB
:1005C0008CC1ADD1CEE1EFF1311210027332522263
:1005D000B5529442F772D662399318837BB35AA30B
:1005E000BDD39CC3FFF3DEE3622443342004011433
:1005F000E664C774A44485546AA54BB5288509955B
:10060000EEE5CFF5ACC58DD5533672261116300602
:10061000D776F6669556B4465BB77AA719973887AA
:10062000DFF7FEE79DD7BCC7C448E5588668A778C2
:100630004008611802282338CCC9EDD98EE9AFF9FA
:10064000488969990AA92BB9F55AD44AB77A966AA2
:10065000711A500A333A122AFDDBDCCBBFFB9EEB4A
:10066000799B588B3BBB1AABA66C877CE44CC55C72
:10067000222C033C600C411CAEED8FFDECCDCDDD9A
:100680002AAD0BBD688D499D977EB66ED55EF44E42
:10069000133E322E511E700E9FFFBEEFDDDFFCCFEA
:1006A0001BBF3AAF599F788F8891A981CAB1EBA13E
:1006B0000CD12DC14EF16FE18010A100C230E320BA
:1006C0000450254046706760B9839893FBA3DAB362
:1006D0003DC31CD37FE35EF3B1029012F322D2320A
:1006E0003542145277625672EAB5CBA5A895898532
:1006F0006EF54FE52CD50DC5E234C324A01481045A
:100700006674476424540544DBA7FAB79987B89701
:100710005FE77EF71DC73CD7D326F2369106B016A9
:1007200057667676154634564CD96DC90EF92FE9C1
:10073000C899E9898AB9ABA94458654806782768F9
:10074000C018E1088238A3287DCB5CDB3FEB1EFBA1
:10075000F98BD89BBBAB9ABB754A545A376A167A49
:10076000F10AD01AB32A923A2EFD0FED6CDD4DCD71
:10077000AABD8BADE89DC98D267C076C645C454C99
:10078000A23C832CE01CC10C1FEF3EFF5DCF7CDF41
:100790009BAFBABFD98FF89F176E367E554E745EE9
:1007A000932EB23ED10EF01E4572726F722025302C
:1007B00032582072656164696E67206461746120DB
:1007C00066726F6D207364206361726420285231F9
:1007D0003D25303258292E0D0A000D0A20204D618A
:1007E0006E7566616374757265722049443A20259E
:1007F000690D0A0020204170706C69636174696F33
:100800006E2049443A2025730D0A00202050726F53
:1008100064756374204E616D653A2025730D0A007E
:10082000202050726F64756374205265762E3A20D2
:1008300025692E25690D0A00202053657269616CB7
:10084000204E6F2E3A200025303258000D0A00202D
:10085000204D616E756661632E20446174653A2097
:1008600025692F25690D0A0D0A000D0A20535343EF
:1008700020696E69742E2E2E006F6B000D0A2053B6
:10088000444320696E69742E2E2E00726573657460
:100890002074696D656F75740042616420636D64D6
:1008A000382052313D253032582E00426164206399
:1008B0006D643820523720636865636B2070617403
:1008C0007465726E2E0D0A00436172642069732094
:1008D000696E636F6D70617469626C6520746F20FE
:1008E000332E33562E0D0A0042616420636D643549
:1008F0003820523120253032782E004E6F7420611E
:100900006E2053442D434152442E004361726420B3
:10091000697320696E636F6D70617469626C6520C4
:10092000746F20332E33562E004261642041636D74
:100930006434312052313D253032582E00496E69E1
:10094000742074696D656F75742E00496E6974202A
:100950006572726F722E004572726F7220736574C9
:1009600074696E6720626C6F636B206C656E677470
:100970006820746F203531322E004572726F7220FC
:1009800072656164696E67204349442E0D0A004513
:1009900072726F722072656164696E67204353449E
:1009A0002E006F6B0D0A000D0A202053442D434189
:1009B00052442056312E78000D0A202053442D43F6
:1009C0004152442056322E30206F72206C61746583
:1009D00072000D0A20204361706163697479203DC3
:1009E000202569204D42004E6F20436172642069CA
:1009F0006E20536C6F742E000D0A20534443206404
:100A000065696E69742E2E2E006F6B004572726FD1
:100A10007220253032582077726974696E672064BD
:100A200061746120746F2073642063617264202894
:100A3000523D25303258292E0D0A000D0A2046411C
:100A400054313620696E69742E2E2E0053442D4386
:100A500061726420636F756C64206E6F74206265D0
:100A600020696E697469616C697A65642E004572EB
:100A7000726F722072656164696E672074686520A8
:100A80004D42522E004572726F7220726561646928
:100A90006E6720746865205642522E005642523AC4
:100AA00020536563746F722073697A65206E6F746A
:100AB00020737570706F727465642E005642523ADE
:100AC00020426164206E756D626572206F662073CE
:100AD0006563746F72732E005642523A20506172F1
:100AE000746974696F6E20697374206E6F74204628
:100AF0004154313620747970652E00202E2E2E6FD1
:100B00006B000D0A2573203C2D2D20256420697370
:100B1000206F7574206F662072616E6765205B259B
:100B2000642E2E2E25645D000D0A2573203C2D2D8C
:100B300020756E6B6E6F776E20706172616D65747B
:100B400065720D0A000D0A2053657474696E67732F
:100B500020696E69742E2E2E004552524F523A2053
:100B60004F70656E696E672073657474696E677324
:100B70002066696C6521006F6B004552524F523AF6
:100B8000204372656174696E672064656661756C87
:100B9000742073657474696E67732066696C65216F
:100BA0000044656661756C742073657474696E6762
:100BB000732066696C6520637265617465642100E9
:100BC0005573696E672064656661756C7420766123
:100BD0006C75657321000D0A4F70656E696E672034
:100BE0006B6D6C2D66696C653A2025730D0A000DDE
:100BF0000A4572726F72206F70656E696E67206B46
:100C00006D6C2D66696C653A2025730D0A000D0A1E
:100C10004572726F722067657474696E67206672C0
:100C20006565206B6D6C2D66696C65206E616D6508
:100C30000D0A000D0A4572726F72206C6F6767694A
:100C40006E6720746F206B6D6C2D66696C650D0A84
:100C5000000D0A436C6F73696E67206B6D6C2D66B7
:100C6000696C650D0A000D0A4572726F7220636C23
:100C70006F73696E67206B6D6C2D66696C650D0A0C
:100C8000000D0A4F70656E696E67206770782D667B
:100C9000696C653A2025730D0A000D0A4572726F62
:100CA00072206F70656E696E67206770782D666957
:100CB0006C653A2025730D0A000D0A4572726F7239
:100CC0002067657474696E67206672656520677059
:100CD000782D66696C65206E616D650D0A000D0AE0
:100CE0004572726F72206C6F6767696E6720746FF0
:100CF000206770782D66696C650D0A000D0A436CDB
:100D00006F73696E67206770782D66696C650D0A70
:100D1000000D0A4572726F7220636C6F73696E67A3
:100D2000206770782D66696C650D0A000D0A3C2FEE
:100D3000636F6F7264696E617465733E0D0A3C2F58
:100D40004C696E65537472696E673E0D0A003C4CC7
:100D5000696E65537472696E673E0D0A3C74657303
:100D600073656C6C6174653E313C2F74657373659B
:100D70006C6C6174653E0D0A3C616C7469747564D9
:100D8000654D6F64653E72656C6174697665546F1C
:100D900047726F756E643C2F616C7469747564651D
:100DA0004D6F64653E0D0A3C636F6F7264696E61DE
:100DB0007465733E0D0A003C2F506C6163656D6174
:100DC000726B3E0D0A003C506C6163656D61726B25
:100DD0003E0D0A3C6E616D653E466F6C6C6F774DE3
:100DE000653C2F6E616D653E0D0A3C7374796C65D0
:100DF00055726C3E23464D5F6770732D7374796C2A
:100E0000653C2F7374796C6555726C3E0D0A003C1D
:100E10002F446F63756D656E743E0D0A3C2F6B6DCC
:100E20006C3E0D0A003C3F786D6C207665727369EC
:100E30006F6E3D22312E302220656E636F64696EC5
:100E4000673D225554462D38223F3E0D0A3C6B6DBE
:100E50006C20786D6C6E733D22687474703A2F2F1D
:100E600065617274682E676F6F676C652E636F6D56
:100E70002F6B6D6C2F322E32223E0D0A3C446F6375
:100E8000756D656E743E0D0A3C6E616D653E4D6913
:100E90006B726F6B6F7074657220475053206C6F6C
:100EA0006767696E673C2F6E616D653E0D0A0D0ABE
:100EB0003C5374796C652069643D22464D5F6770D0
:100EC000732D7374796C65223E0D0A3C4C696E6516
:100ED0005374796C653E0D0A3C636F6C6F723E66AD
:100EE000663030666630303C2F636F6C6F723E0D3B
:100EF0000A3C77696474683E323C2F776964746891
:100F00003E0D0A3C2F4C696E655374796C653E0D3D
:100F10000A3C2F5374796C653E0D0A003C2F7472A5
:100F20006B7365673E0D0A003C74726B7365673EB8
:100F30000D0A003C2F74726B3E0D0A003C74726BFC
:100F40003E0D0A3C6E616D653E466F6C6C6F774D71
:100F5000653C2F6E616D653E0D0A003C2F67707811
:100F60003E0D0A003C3F786D6C2076657273696FA8
:100F70006E3D22312E302220656E636F64696E678C
:100F80003D225554462D3822207374616E64616C85
:100F90006F6E653D226E6F22203F3E0D0A3C6770EA
:100FA000782063726561746F723D22466F6C6C6F5E
:100FB000774D65222076657273696F6E3D22312E02
:100FC0003022203E0D0A0D0A3C6D65746164617427
:100FD000613E0D0A3C6C696E6B20687265663D224D
:100FE000687474703A2F2F7777772E6D696B726FF4
:100FF0006B6F707465722E6465223E0D0A3C7465D9
:1010000078743E4D696B726F4B6F707465723C2FD4
:10101000746578743E0D0A3C2F6C696E6B3E0D0A48
:101020003C2F6D657461646174613E0D0A0D0A00A8
:1010300011241FBECFEFD0E1DEBFCDBF13E0A0E093
:10104000B1E0EAEFF5E802C005900D92AE39B107C4
:10105000D9F71DE0AEE9B3E001C01D92A335B10799
:10106000E1F70C9435080C940000CFEFD0E1DEBF1F
:10107000CDBF84B7877F84BF8091600088618093F3
:101080006000109260000E942A1728980E94C912DE
:101090000E94360A0E94BA180E94270F0E94CF1A97
:1010A0000E94B51B78940E94142E0E94BA330E94AD
:1010B000F437289A29988CE790E09F938F931F929A
:1010C0000E9434100F900F900F9085E690E09F9350
:1010D0008F9381E090E09F938F931F921F928EE8F1
:1010E00090E09F938F931F920E9434108DB79EB70C
:1010F00009960FB6F8949EBF0FBE8DBF8EEA90E0A2
:101100009F938F931F920E9434100F900F900F9017
:101110008FEC90E09F938F931F920E9434100E9457
:101120006A1388EE93E00E9449139093AA03809378
:10113000A9030F900F900F900E9476320E941938E9
:101140000E94D41B882309F42BC188EC90E0909373
:10115000BF038093BE0320919E03822F992701979E
:1011600009F441C121E020939E03822F9927909397
:10117000D6058093D5058130910509F41DC10297EC
:1011800009F43AC181E080939E038091C0018823D5
:1011900009F4F2C08091B4069091B5069093C4050D
:1011A0008093C3058091B2069091B3069093C605D3
:1011B0008093C5058091A8069091A9069093C805D3
:1011C0008093C7058091AA069091AB069093CA05BB
:1011D0008093C9058091B0069091B1069093CC059B
:1011E0008093CB058091A6069091A7069093CE059B
:1011F0008093CD058091AC069091AD069093D0057B
:101200008093CF058091AE069091AF069093D20562
:101210008093D10580910001909101019C01220FE2
:10122000331F280F391F8091B0069091B10600241A
:10123000969587950794969587950794982F802D76
:1012400060E771E00E949942260F371F3695279577
:101250003695279530930101209300013093D405F2
:101260002093D3054091A5035091A6034436510520
:101270000CF0B1C0253531050CF0B2C0E2E0F0E071
:10128000F093A803E093A7034F5F5F4F5093A6032B
:101290004093A503F093E405E093E3055093E6053E
:1012A0004093E5056091A3037091A4036E177F0737
:1012B0000CF086C0443651050CF482C0A091BE03E8
:1012C000B091BF03109709F07BC08091A10390916A
:1012D000A203C3E0893E9C078CF084E690E09093E3
:1012E000BF038093BE036F5F7F4F7093A40360932F
:1012F000A303B093A203A093A103CD0165E08C3DAD
:1013000096072CF401969093A2038093A103EE0F0D
:10131000FF1FE295F295F07FFE27E07FFE272E1754
:101320003F0724F02A3431050CF04FC044365105F4
:101330000CF44BC080E093E090930601809305018C
:101340008091BE039091BF03892B31F480E797E130
:101350009093BF038093BE0380919F039091A0035D
:1013600082609093A00380939F031092C0018091AC
:101370007A00886C80937A000E94170D0E94AE0D4F
:1013800080919F039091A003892BC1F028980E941F
:1013900076320E9419380E94D41B882309F0D5CEDA
:1013A00020919E03822F99279093D6058093D5058F
:1013B0008130910509F0E3CE2998E7CE289ABCCE7A
:1013C0008091A1039091A20399CF80919F03909166
:1013D000A0038D7FC6CFE091A703F091A8035ACF59
:1013E000E3E0F0E04DCF80919F039091A003892B23
:1013F00009F0BBCE22E0B7CE8091A9039091AA0359
:101400000E945213882309F4C0CEC0919A05C130BE
:1014100069F08AEF90E00E9449139093AA038093A9
:10142000A90385B192E0892785B9AFCE88EE93E014
:101430000E9449139093AA038093A9038FEF9FEF13
:1014400090939C0580939B05C0939D058CE38093AE
:101450009E0510929F051092A0051092A105109272
:10146000A2051092A305C093B303DBCFCF93CFB7F0
:101470002AE230E0F8948091C1008F778093C10018
:101480008091C1008F7B8093C100589A5098599ADF
:10149000519A832F99278093C5002093C40080918F
:1014A000C00082608093C00088E18093C100809179
:1014B000C2008F778093C2008091C2008F7B80939F
:1014C000C2008091C2008F7D8093C2008091C200D3
:1014D0008F7E8093C2008091C200877F8093C2007C
:1014E0008091C1008B7F8093C1008091C200846095
:1014F0008093C2008091C20082608093C20080917C
:10150000C00087FF0CC08091C6008091C000882376
:1015100034F48091C6008091C0008823A4F38091A8
:10152000C10080688093C1008091C1008064809375
:10153000C1008091AB039091AC030E94491390933A
:101540009A06809399061092B1031092AF031092FD
:10155000AE031092AD0381E0809303011092AC05BD
:101560008093AD0584E08093B0058AE08093AE055A
:101570001092AF05CFBF789482ED92E09F938F9346
:101580001F920E9434100F900F900F90CF910895EA
:101590001F920F920FB60F9211248F939F93EF9388
:1015A000FF93809103018823A9F48091B90390915E
:1015B000BA030196FC01ED5FF94FE081ED3079F05F
:1015C0008639910561F09093BA038093B903E09353
:1015D000C6000EC01092BA031092B90309C010924F
:1015E000BA031092B90381E080930301E093C6002F
:1015F000FF91EF919F918F910F900FBE0F901F90D1
:1016000018951F920F920FB60F9211242F933F93AC
:101610004F935F938F939F93AF93BF93CF93DF933A
:10162000EF93FF935091C6008091B103882309F096
:1016300073C04091BD034423B9F45332E1F05D30EF
:1016400011F1E42FFF27E850FB4F50834F5F409389
:10165000BD038091BB039091BC03850F911D9093B6
:10166000BC038093BB0358C0463948F38093BD0345
:101670008093B10351C05093F80481E08093BD037F
:1016800083E290E0ECCFA42FBB27A850BB4FFD0115
:10169000329780812091BB033091BC03281B310914
:1016A000ED0121978881281B3109C9019F70909312
:1016B000BC038093BB030024880F991F001C880F74
:1016C000991F001C892F902D982F935C2F733070D9
:1016D000235C8081891729F01092B1031092BD0319
:1016E0001BC088818217C1F75C934F5F4093B003A2
:1016F00081E08093B1038091FA04823579F788E123
:1017000090E02CE00FB6F894A895809360000FBE8F
:10171000209360001092BD03FF91EF91DF91CF9174
:10172000BF91AF919F918F915F914F913F912F9179
:101730000F900FBE0F901F901895AC01A0E0B0E085
:101740009D01A817B90748F4E3E0F6E08191280F5E
:10175000311D1196A417B507C8F33F70FD01ED5F69
:10176000F94FC9010024880F991F001C880F991F89
:10177000001C892F902D835C80831196FD01ED5F05
:10178000F94F2F733070822F835C8083AC5FB94F29
:101790008DE08C9310920301809103068093C60024
:1017A0000895BF92CF92DF92EF92FF920F931F9313
:1017B000CF93DF93CDB7DEB72C859D857E85BB2487
:1017C00083E2809303069F599093040620930506B5
:1017D00003E010E0772309F4ADC0CF84D88843E15B
:1017E000E42EF12CEC0EFD1EA989BA8971501097D8
:1017F00009F4A0C0109709F43CC0F601EB0DF11DEF
:10180000B3949081119789F47723A1F1F70122E035
:1018100030E0E20EF31ED701C080D180E20EF31E4D
:101820000D90BC91A02DBB247150109719F1F601B9
:10183000EB0DF11DB3944081119709F466C0109728
:10184000D1F0F601EB0DF11DB39460811197A1F475
:10185000772391F0F7013296D701CD90DC9032E0FA
:10186000E32EF12CEE0EFF1EA081B181BB2471503E
:1018700003C090E040E060E0F801ED5FF94F892F90
:1018800086958695835C80830F5F1F4FF801ED5F1F
:10189000F94F892F99278370907082959295907F48
:1018A0009827807F982755279A01329522952F7087
:1018B00023273F702327822B835C80830F5F1F4F7A
:1018C000F801ED5FF94F4F705070440F551F440FF2
:1018D000551F862F99270024880F991F001C880FF9
:1018E000991F001C892F902D842B835C80830F5FB0
:1018F0001F4FF801ED5FF94F6F73635C60830F5FFB
:101900001F4F109709F076CF15C0772309F4B3CF96
:10191000F701A2E0B0E0EA0EFB1ED701C080D18043
:1019200022E030E0E20EF31E0D90BC91A02DBB240E
:10193000715085CFC8010E949D0BDF91CF911F91FF
:101940000F91FF90EF90DF90CF90BF900895A3E0AC
:101950007A2F4091B003465009F45FC0E72FFF276C
:10196000E850FB4F80818D537F5FE72FFF27E850C2
:10197000FB4F20812D537F5FE72FFF27E850FB4F60
:1019800030813D537F5FE72FFF27E850FB4F608199
:101990006D537F5F9927880F991F880F991F522FCA
:1019A00052955F70582B822F99278F709070829577
:1019B0009295907F9827807F9827232F26952695AC
:1019C000282B832F992783709070002496958795F4
:1019D0000794969587950794982F802D682B4150F2
:1019E0004F3FD9F0EA2FFF27E850FB4F5083AF5FFE
:1019F00041504F3F91F0EA2FFF27E850FB4F2083E3
:101A0000AF5F41504F3F49F0EA2FFF27E850FB4FAF
:101A10006083AF5F442309F0A1CF8BEF94E09093F4
:101A2000AF038093AE03A350A093AD0308958091BC
:101A3000B103882309F408950E94A70C8091F9044A
:101A40008B36E1F18091FA0499278736910591F15F
:101A5000883691058CF48136910509F447C08436A7
:101A6000910509F451C01092AF031092AE03109289
:101A7000AD031092B10308958C36910549F18D366E
:101A80009105FCF48836910571F78FEF8093020180
:101A9000E091AE03F091AF0380819091C403892B54
:101AA0008093C403882311F01092B20381E08093E5
:101AB000B703D9CF81E08093B503D5CF8091FA04E5
:101AC000C1CF8637910579F681E08093B803CBCFFB
:101AD0008FEF80930201E091AE03F091AF0380811C
:101AE0008093C50381E08093B603BDCFE091AE0340
:101AF000F091AF03E081E032D8F08FE180930401F0
:101B00008FEF80930201AFCFE091AE03F091AF036E
:101B100090818AE0989FC00111249093AC03809338
:101B2000AB03892B09F49FCF81E08093B4039BCF53
:101B3000E0930401E5CFCF93C82F8A3029F080913C
:101B4000C00085FFFCCF04C08DE00E949B0DF7CF45
:101B5000C093C60080E090E0CF9108951F93CF938B
:101B6000DF93CDB7DEB760970FB6F894DEBF0FBE38
:101B7000CDBF80910301882309F45FC18091B80330
:101B8000882309F06EC08091B703882329F08091E3
:101B90000301882309F0E9C08091B603882329F066
:101BA00080910301882309F0B5C0809104018F3F23
:101BB000A1F1992782959295907F9827807F982709
:101BC0008E529F4F40E150E0BC01CE0101960E9431
:101BD000D23E80E190E09F938F93CE0101969F9338
:101BE0008F9381E090E09F938F9384E091E09F93A7
:101BF0008F9382E08F938AE08F9381E48F930E948A
:101C0000D10B8FEF809304012DB73EB7255F3F4F77
:101C10000FB6F8943EBF0FBE2DBF8091B503882349
:101C200029F080910301882309F059C08091AB030A
:101C30009091AC03892B09F0CBC08091B403882329
:101C400029F080910301882309F0CCC08091B3036F
:101C5000882309F4F2C080910301882309F4EDC0C0
:101C600021C080910301882309F48DCF8AE090E0A0
:101C70009F938F938CEA95E09F938F9381E08F934E
:101C80008AE08F9386E58F930E94D10B1092B80360
:101C90002DB73EB7295F3F4F0FB6F8943EBF0FBE3A
:101CA0002DBF71CF8EE190E09F938F938EE895E0EA
:101CB0009F938F9381E08F9312E01F9383E78F931D
:101CC0000E94D10B10939A051092B3038DB79EB763
:101CD00007960FB6F8949EBF0FBE8DBFAEC08BE0C7
:101CE00090E09F938F9386EB95E09F938F9381E095
:101CF0008F938AE08F9387E48F930E94D10B109289
:101D0000B5038DB79EB707960FB6F8949EBF0FBE6A
:101D10008DBF8CCF0E94731380E590E09F938F93CB
:101D200087E091E09F938F9321E030E03F932F93E2
:101D300087E591E09F938F933F932F9385EC93E0FA
:101D40009F938F9383E08F938AE08F938CE48F939C
:101D50000E94D10B1092B6038DB79EB70F960FB6A7
:101D6000F8949EBF0FBE8DBF20CF0E94731384E1F5
:101D700090E09F938F939091B20384E1989FC0016C
:101D80001124895F9E4F9F938F9381E090E09F93F2
:101D90008F9382EB93E09F938F9382E08F938AE0FF
:101DA0008F9388E48F930E94D10B8091B2038F5F51
:101DB0002DB73EB7255F3F4F0FB6F8943EBF0FBE1D
:101DC0002DBF8430A8F11092B2031092B703E4CE75
:101DD0008091990690919A060E945213882309F0E7
:101DE00030CF2BCF82E490E09F938F9381EC95E0EE
:101DF0009F938F9381E08F938AE08F9384E48F93F6
:101E00000E94D10B8091AB039091AC030E944913C7
:101E100090939A06809399061092B4032DB73EB71B
:101E2000295F3F4F0FB6F8943EBF0FBE2DBF0ECFB8
:101E30008093B2031092B703AFCE60960FB6F894BA
:101E4000DEBF0FBECDBFDF91CF911F91089585EE0C
:101E500092E09F938F931F920E9434104FB72AE213
:101E600030E0F8948091C9008F778093C900809109
:101E7000C9008F7B8093C9008091C9008F7D8093BA
:101E8000C9005A9A52985B9A539A832F9927809344
:101E9000CD002093CC008091C80082608093C80060
:101EA00088E18093C9008091CA008F778093CA002F
:101EB0008091CA008F7B8093CA008091CA008F7D79
:101EC0008093CA008091CA008F7E8093CA0080915F
:101ED000CA00877F8093CA008091C9008B7F80935E
:101EE000C9008091CA0084608093CA008091CA00B2
:101EF00082608093CA000F900F900F908091C8006D
:101F000087FF0CC08091CE008091C800882334F4F4
:101F10008091CE008091C8008823A4F38091C900ED
:101F200080688093C9008091C90080648093C90053
:101F30004FBF789486EF92E09F938F931F920E94F9
:101F400034100F900F900F9008951F920F920FB6BC
:101F50000F9211242F933F934F935F936F937F932F
:101F60008F939F93AF93BF93EF93FF938091CE0096
:101F70000E94D619FF91EF91BF91AF919F918F91E0
:101F80007F916F915F914F913F912F910F900FBE75
:101F90000F901F901895982F80919B06813031F0FB
:101FA000892F0E949B0D282F33270CC08091C303DB
:101FB000E82FFF27E95FFE4F90838F5F8093C30375
:101FC00021E030E0C90108950F931F93CF93DF9371
:101FD0008C01EB01672B71F0F80181918F010E9458
:101FE000CB0F219739F0F80181918F010E94CB0F1F
:101FF000219791F7DF91CF911F910F9108950F9342
:102000001F93CF93DF938C01EB01672B81F0F801D5
:102010000F5F1F4F84910E94CB0F219741F0F80171
:102020000F5F1F4F84910E94CB0F219781F7DF91A3
:10203000CF911F910F910895CF93C82F181634F4A4
:1020400080E20E94CB0FC1501C16D4F3CF910895AB
:10205000CF93C82F181634F480E30E94CB0FC150E1
:102060001C16D4F3CF9108952F923F924F925F9216
:102070006F927F928F929F92AF92BF92CF92DF9298
:10208000EF92FF920F931F93CF93DF93CDB7DEB7FD
:10209000E0970FB6F894DEBF0FBECDBF26968FAD8A
:1020A00026972896EEADFFAD2897882499245401F1
:1020B00080939B0648E4C42ED12CCC0EDD1E7F01FC
:1020C000C701F7011491112331F0153221F0089462
:1020D000E11CF11CF6CFB701681B790B09F095C024
:1020E000112309F43DC20894E11CF11C1FA63FA472
:1020F000232C0FEF39A6F7010894E11CF11C149171
:102100001537C9F1812F80628837A9F1103209F49F
:1021100040C0133209F48DC01A3209F479C01D325F
:1021200009F476C01B32C9F11E32C9F1103309F42B
:102130008AC0812F8153893008F07EC060E070E052
:10214000CB01880F991F880F991F880F991F860F41
:10215000971F680F791F610F711D60537040F70161
:102160000894E11CF11C1491812F80538A3040F3B4
:10217000262E153739F630FE3DC0F60184E090E09A
:10218000C80ED91E80809180A280B380103209F0E1
:10219000C0CF89A5882309F0AECF19A7ACCFF7012E
:1021A0000894E11CF11C14911A3209F451C060E04A
:1021B00070E014C0CB01880F991F880F991F880FFA
:1021C000991F860F971F680F791F610F711D60534C
:1021D0007040F7010894E11CF11C1491812F805389
:1021E0008A3040F3EFEF6F3F7E0714F46FEF7FEF1D
:1021F000062F86CFF60182E090E0C80ED91E8081BE
:1022000091814C01AA24BB2481CF0E94FF0F68CF8B
:102210001A3251F4F60182E090E0C80ED91E2080F7
:1022200022200CF068CF219490E1392AEFED3E2274
:1022300062CF98E0392A5FCF1836C9F01C36D1F446
:1022400081E0382A58CF34FC56CFF0E23F2A53CFF2
:10225000F60182E090E0C80ED91E608171819FEF87
:102260006F3F790714F46FEF7FEF062F44CF24E020
:10227000322A41CF133609F44DC1143409F41FC179
:10228000143609F41CC1193609F419C11F3409F4B4
:102290000FC11F3609F40CC1103709F4F9C0133708
:1022A00009F4B2C0153509F4ECC0153709F4E9C0DA
:1022B000183509F444C0183709F441C0112309F452
:1022C0004FC1CE0101969DA78CA7198381E0482EAE
:1022D00019A6632C7724042D5FA4541857FC2DC035
:1022E00029A5222331F10F5F050DC3018073907082
:1022F000892B09F42FC1222309F027C166FC1BC1D9
:10230000C30180739070809709F410C1852D0E94DD
:102310002810842D992787FD9095BC018CA59DA53B
:102320000E94E40F64FECCCE822D801B0E941C1004
:10233000C7CE66FED9CF0E5FD7CF5524D1CFE0E10F
:10234000EEA733FE07C081149104A104B10411F07B
:10235000F0E43F2A19A60FA707FD02C02FED322295
:10236000CE0189969DA78CA781149104A104B10484
:1023700019F49FA5992361F1EEA54E2E55246624EC
:10238000772418AA84149504A604B70410F0F1E089
:10239000F8ABC501B401A30192010E94C042DC0167
:1023A000CB01082F8A30F0F4005DECA5FDA5029367
:1023B000FDA7ECA7C501B401A30192010E94C04290
:1023C00049015A01F8A9FF23E1F62EA5283079F03A
:1023D000632C7724CE010196482EFCA54F1A28E2E3
:1023E000420E79CF095A183501F70F7DDECF632CE5
:1023F000772463FEEFCF003369F380E3ECA5FDA5FE
:102400008293FDA7ECA7E6CFF60182E090E0C80E2C
:10241000D91E0190F081E02DFDA7ECA7EF2B81F4F0
:10242000FE013196FDA7ECA788E289838EE68183C1
:1024300085E78B838CE68C838D8389E28E831F8274
:1024400007FD15C0802F992787FD9095AC0160E0AE
:1024500070E08CA59DA50E94DF3E009731F0482ECC
:10246000FCA54F1A04150CF033CF402E31CFECA54C
:10247000FDA501900020E9F731974E2E2CA5421AB8
:1024800027CF153511F481E0382A9AE09EA762CF54
:10249000F60182E090E0C80ED91E808191814C0146
:1024A000AA24BB2490E19EA7E0E43E2A18E752CF7D
:1024B0001F3411F4E1E03E2AF8E0FEA74BCF1434BC
:1024C00011F491E0392A30FE18C0F60184E090E062
:1024D000C80ED91E80809180A280B380B7FE0AC04A
:1024E000B094A09490948094811C911CA11CB11C68
:1024F0008DE289A79AE09EA72ECFF60182E090E0B8
:10250000C80ED91E808191814C01AA2497FCA09409
:10251000BA2CE4CFFE013196FDA7ECA7F60182E0CC
:1025200090E0C80ED91E80818983D0CE822D801B79
:102530000E942810EBCE80E38AA71BA762E070E020
:10254000CE018A960E94E40FDBCE61E070E0CE01FE
:102550008996F8CF822D801B0E941C1029A5CBCE16
:10256000E0960FB6F894DEBF0FBECDBFDF91CF91DE
:102570001F910F91FF90EF90DF90CF90BF90AF90A1
:102580009F908F907F906F905F904F903F902F9093
:1025900008959FB7F8943F9A479884B58C7084BD8E
:1025A00085B5877385BD85B5887F826085BD16BC7E
:1025B00080916E00897F80936E0080916E008160B3
:1025C00080936E0010929D0610929C0610929E06BB
:1025D00010929F061092A0061092A1061092A206D9
:1025E0001092A4061092A3061092A5061092C103A1
:1025F0001092C0039FBF789408951F920F920FB658
:102600000F9211242F933F938F939F938091C20336
:1026100081508F3F41F18093C2038091BE0390911E
:10262000BF03892BB9F08091BE039091BF0301973E
:102630009093BF038093BE038091BE039091BF032C
:10264000209105013091060182239323892B49F4BF
:10265000479816C08FEF9FEF909306018093050176
:10266000F7CF479A0DC089E08093C2038091C003E1
:102670009091C10301969093C1038093C003CDCF85
:102680009F918F913F912F910F900FBE0F901F90B0
:1026900018952091C0033091C103280F391FC9013B
:1026A000019708952091C0033091C103821B930BC1
:1026B000892F990F990B80780895CF93DF930E940B
:1026C0004913EC01CE010E9452138823D9F3DF9104
:1026D000CF91089590E2E7E0F1E08FE4919381508B
:1026E00087FFFCCF0895BF92CF92DF92EF92FF92C7
:1026F0000F931F93CF93DF932091C40320FF08C053
:102700008091C503882309F45BC081508093C50381
:1027100021FF0AC09091C50380915701981709F4D1
:10272000F5C19F5F9093C503822F992780FF02C058
:1027300081FD43C00E946A139091C50380915701A7
:10274000891718F48093C503982F9A3060F581E1BA
:102750008093C303892F99279F938F9389EF92E0EA
:102760009F938F9381E08F930E9434100F900F906E
:102770000F900F900F909091C503C92FDD27C130A6
:10278000D10519F1C230D1050CF4C3C1C230D10555
:1027900009F454C1239709F43DC291509093570115
:1027A0001092C5034BC380E18093C303892F9927FF
:1027B0009F938F938EEF92E0D3CF1092C503BACF41
:1027C000809157018093C503A3CF8091F2038823A2
:1027D00009F4DEC18091D50399278230910509F46F
:1027E0005AC2833091050CF008C2892B09F408C342
:1027F0001092C3038091D40399279F938F938AEB00
:1028000093E09F938F9381E08F930E9434100F90F9
:102810000F900F900F900F90E090C603F090C703B9
:102820000091C8031091C90317FDC3C24BE2B42E37
:10283000C801B70120E836E948E950E00E94E242C9
:10284000690137FDB1C2C801B70120E836E948E99E
:1028500050E00E94E242DC01CB01BC01CD0120E14D
:1028600037E240E050E00E94E242E90137FDC4C295
:10287000C801B70120E836E948E950E00E94E24289
:10288000DC01CB01BC01CD0120E137E240E050E0AA
:102890000E94E242DC01CB01BC01CD012AE030E024
:1028A00040E050E00E94E242DA01C90197FDA0C277
:1028B00084E18093C3033F932F93DF93CF93DF9201
:1028C000CF928B2D99279F938F938DEC93E09F93BD
:1028D0008F9381E08F930E943410E090CA03F090B0
:1028E000CB030091CC031091CD038DB79EB70B960F
:1028F0000FB6F8949EBF0FBE8DBF17FD76C22BE2B8
:10290000B22EC801B70120E836E948E950E00E943C
:10291000E242690137FD64C2C801B70120E836E927
:1029200048E950E00E94E242DC01CB01BC01CD014C
:1029300020E137E240E050E00E94E242E90137FD49
:102940004BC2C801B70120E836E948E950E00E94CF
:10295000E242DC01CB01BC01CD0120E137E240E0E5
:1029600050E00E94E242DC01CB01BC01CD012AE033
:1029700030E040E050E00E94E242DA01C90197FDF8
:1029800027C288E28093C3033F932F93DF93CF93B3
:10299000DF92CF928B2D99279F938F9384EE93E0B4
:1029A0009F938F9381E08F930E943410E090CE0329
:1029B000F090CF030091D0031091D1038DB79EB753
:1029C0000B960FB6F8949EBF0FBE8DBF17FDFDC1CD
:1029D0008BE2B82EC801B70128EE33E040E050E0AA
:1029E0000E94E242690137FDEBC1C801B70128EE40
:1029F00033E040E050E00E94E242DC01CB01EC0118
:102A000097FDDAC18CE38093C303DF93CF93DF920A
:102A1000CF928B2D99279F938F938BEF93E09F936A
:102A20008F9381E08F930E9434108DB79EB70996E3
:102A30000FB6F8949EBF0FBE8DBF00C28091F20307
:102A4000882309F484C18091D503992782309105A8
:102A500009F4E0C1833091050CF410C1039709F427
:102A6000E3C11092C3038091D40399279F938F935E
:102A700083E994E09F938F9381E08F930E943410B9
:102A80000F900F900F900F900F9084E18093C303ED
:102A90008091DA039091DB039F938F9386EA94E011
:102AA0009F938F9311E01F930E94341088E28093CC
:102AB000C3030F900F900F900F900F908091DE0343
:102AC0009091DF039F938F9389EB94E09F938F9373
:102AD0001F930E9434108CE38093C3030F900F90D8
:102AE0000F900F900F908091E2039091E3039F93DA
:102AF0008F938CEC94E09F938F931F930E943410DC
:102B00000F900F900F900F900F9098C11092C503E7
:102B10000BCE209709F041CE1092C30383E093E0DF
:102B20009F938F9311E01F930E94341084E1809350
:102B3000C3030F900F900F9081E193E09F938F93C9
:102B40001F930E94341088E28093C3030F900F906C
:102B50000F9085E690E09F938F9381E090E09F93A4
:102B60008F93DF93CF938FE193E09F938F931F9386
:102B70000E9434108CE38093C3038DB79EB70996EF
:102B80000FB6F8949EBF0FBE8DBF8BE293E02CC0B2
:102B90008093C30386E393E09F938F9311E01F9389
:102BA0000E94341084E18093C3030F900F900F9024
:102BB00082E493E09F938F931F930E94341088E2E6
:102BC0008093C3030F900F900F9087E593E09F933E
:102BD0008F931F930E9434108CE38093C3030F9054
:102BE0000F900F908CE693E09F938F931F930E941A
:102BF00034100F900F900F9021C1039709F0F8CD7A
:102C00001092C3038091D40399279F938F9387EAEF
:102C100093E0F7CD1092C3038FED94E09F938F93D1
:102C2000C1E0CF930E9434100F900F900F908091CD
:102C3000A5068823D1F584E18093C3038CEE94E04C
:102C40009F938F93CF930E94341088E28093C303A5
:102C50000F900F900F9081E095E09F938F93CF930B
:102C60000E9434108CE38093C3030F900F900F9059
:102C700086E195E09F938F93CF93B9CF892B09F08D
:102C8000F0CE1092C3038091D40399279F938F9322
:102C90008AE594E0EFCE1092C3038091D403992784
:102CA0009F938F9384E993E0ACCD84E18093C30339
:102CB0008BE295E09F938F93CF930E94341088E22C
:102CC0008093C3030F900F900F9080919C0690917A
:102CD0009D069F938F9380919F0699279F938F9333
:102CE00080919E0699279F938F9380E495E09F9310
:102CF0008F93CF930E9434108CE38093C3038DB7DE
:102D00009EB709960FB6F8949EBF0FBE8DBF8091F7
:102D1000A3069091A4069F938F938091A206992772
:102D20009F938F938091A10699279F938F93809172
:102D3000A00699279F938F9385E595E09F938F93A6
:102D4000CF930E9434108DB79EB70B9671CE8093AF
:102D5000C3038FE094E09F938F9311E01F930E9431
:102D6000341084E18093C3030F900F900F908BE198
:102D700094E09F938F931F930E94341088E2809376
:102D8000C3030F900F900F9080E394E09F938F9375
:102D90001F930E9434108CE38093C3030F900F9015
:102DA0000F9085E494E020CFD094C194D108D394BF
:102DB0004ACD5DE2B52E3CCDD095C195DF4F22CEF8
:102DC000D094C194D108D39410CE9DE2B92E02CEF6
:102DD000309521953F4FD5CDD095C195DF4FB1CDE1
:102DE000D094C194D108D39497CD3DE2B32E89CD30
:102DF000309521953F4F5CCDD095C195DF4F38CDB3
:102E00001092C3038091D40399279F938F9381E8F5
:102E100093E0F7CC1092C3038091D40399279F933A
:102E20008F938DE694E026CE1092C3038091D40355
:102E300099279F938F9380E894E01CCE1092C4034F
:102E4000DF91CF911F910F91FF90EF90DF90CF9086
:102E5000BF900895209A299A219A289A08959C0152
:102E600060E971E00E949942892B61F0C901837089
:102E70009070892B51F4C90164E670E00E94994278
:102E8000892B19F081E090E0089580E090E00895AA
:102E90008F929F92AF92BF92CF92DF92EF92FF926A
:102EA0000F931F93CF93DF934C0180916B04882382
:102EB00021F08091420482FD03C0F40111864DC1CE
:102EC0008091420483FFF9CF8091370490913804B8
:102ED000A0913904B0913A04BC01CD0128EE33E051
:102EE00040E050E00E94C04259016A0180913F04D5
:102EF00090914004AA2797FDA095BA2F2FE0A21623
:102F0000B104C104D10408F01FC10197A109B1099E
:102F100041E75AE369E070E0A40EB51EC61ED71E55
:102F20007C018D0123E0EE0CFF1C001F111F2A9570
:102F3000D1F7E81AF90A0A0B1B0B23E837E04BE03C
:102F400050E0E20EF31E041F151FC601B50120E874
:102F500031E541E050E00E94C042E20EF31E041F42
:102F6000151FC801B70121EB3AE342E050E00E948F
:102F7000C04280E991E0289FE001299FD00D389F51
:102F8000D00D11242196C801B70121EB3AE342E0AC
:102F900050E00E94C0427B018C012CEA3EE840E0F8
:102FA00050E00E94C04284E690E0289FB001299F33
:102FB000700D389F700D1124C60FD71FC801B701BF
:102FC0002CEA3EE840E050E00E94C0427B018C01C8
:102FD00025EB35E040E050E00E94C042A901440FDB
:102FE000551F440F551FC40FD51FC801B70125EB4E
:102FF00035E040E050E00E94C0427B018C0177E464
:10300000E71674E0F70670E0070770E0170708F0AE
:1030100098C0C801B7012DE631E040E050E00E94C1
:10302000C042A9019E01240F351FD4012D933C936A
:103030008DE691E0489FE001499FD00D589FD00D4B
:103040001124CE01AA27BB27E81AF90A0A0B1B0B89
:103050000894E11CF11C011D111DC9010E942F17CC
:10306000882309F46BC04CE851E020E0E22FFF27F1
:10307000EE0FFF1FEE0FFF1FE40FF51F8081918100
:10308000A281B3818E159F05A007B10788F48481C2
:103090009581A681B7818E159F05A007B10740F0E5
:1030A0002F5FE4012A838081EE2DE81BEB832CE067
:1030B0002F5F2C30D8F2C601B50120E831E541E0A0
:1030C00050E00E94C0425B016C0120E13EE040E024
:1030D00050E00E94C042E4012C83C601B50120E10A
:1030E0003EE040E050E00E94C0425B016C012CE3F6
:1030F00030E040E050E00E94C0422D83C601B5019F
:103100002CE330E040E050E00E94C0426E838091AA
:10311000370490913804A0913904B0913A04BC016D
:10312000CD0128EE33E040E050E00E94C042DC01D7
:10313000CB0198878F8381E089870FC048E551E0F4
:1031400094CF43E050E06ECFC1EFDFEFEFEFFFEF42
:10315000AC0EBD1ECE1EDF1EE3CEDF91CF911F91C0
:103160000F91FF90EF90DF90CF90BF90AF909F9026
:103170008F9008958FE695E09F938F931F920E9402
:10318000341010926B0410923604109219041092AD
:10319000F2030F900F900F908EE795E09F938F931F
:1031A0001F920E9434100F900F900F900895CF93AC
:1031B00080916C0490916D040E9452138823D9F081
:1031C00010926E0484E690E00E94491390936D047F
:1031D00080936C0480916E04823008F4E5C0809185
:1031E0006B04813071F082E080936B04809336042D
:1031F00080931904D9C080916E048F5F80936E0410
:10320000E1CF80913604813071F7C0911904C1304B
:1032100051F78091F3039091F40301969093F40396
:103220008093F3038091F2038130E9F21092F2036C
:10323000809142048093D303809166048093D403E9
:10324000809141048093D50380914F049091500464
:10325000A0915104B09152048093D6039093D70368
:10326000A093D803B093D90380915F049091600438
:10327000A0916104B09162048093EE039093EF03F8
:10328000A093F003B093F1038CE996E00E944817F5
:1032900080911E0490911F04A0912004B0912104FC
:1032A0008093C6039093C703A093C803B093C90348
:1032B0008091220490912304A0912404B0912504CC
:1032C0008093CA039093CB03A093CC03B093CD0318
:1032D00080912A0490912B04A0912C04B0912D048C
:1032E0008093CE039093CF03A093D003B093D103E8
:1032F000C093D2038091FD039091FE03A091FF0340
:10330000B09100048093DE039093DF03A093E00369
:10331000B093E1038091F9039091FA03A091FB032C
:10332000B091FC038093DA039093DB03A093DC035A
:10333000B093DD038091010490910204A0910304F5
:10334000B0910404B095A095909581959F4FAF4F93
:10335000BF4F8093E2039093E303A093E403B09301
:10336000E5038091090490910A04A0910B04B091A7
:103370000C048093E6039093E703A093E803B093D3
:10338000E90380910D0490910E04A0910F04B09177
:1033900010048093EA039093EB03A093EC03B093A3
:1033A000ED03C093F2031FCFCF910895482F2091D2
:1033B0006F04822F99278430910569F1853091053A
:1033C00094F48130910509F466C0823091050CF4C3
:1033D0005BC08230910509F48CC0039709F48DC05D
:1033E00010926F0408958630910509F45AC0863012
:1033F00091052CF18730910509F4A7C0089781F752
:1034000080917304481709F4C1C0E0917804F091E9
:103410007904108243C0842F99279093710480937C
:10342000700490917204940F9093720480917304CD
:10343000890F8093730485E080936F040895842F2F
:103440009927982F88272091700430917104820F5A
:10345000931F909371048093700490917204940F61
:103460009093720480917304890F80937304E091A8
:103470007804F09179048081813009F46FC0108262
:1034800086E080936F040895892B09F0A9CF453B0E
:1034900029F481E0D1CF423609F45EC010926F0466
:1034A0000895E0917404F0917504809176049091F0
:1034B0007704E817F90790F74193F0937504E093C8
:1034C000740490917204940F909372048091730429
:1034D000890F809373048091700490917104019717
:1034E0009093710480937004892B09F07BCF87E05F
:1034F000A3CF413099F683E09FCF842F9927863060
:103500009105E1F18730910574F5029739F68AE16A
:1035100094E090937504809374044D96909377048F
:103520008093760401979093790480937804222302
:1035300009F458CF84E080936F04842F8F5F8093C9
:1035400072048F5F8093730408958091720448170A
:1035500009F05BCF88E070CF82E06ECF10926F04ED
:103560000E94D7180895429709F098CF85EF93E00D
:1035700090937504809374048596D0CF87E394E08C
:103580009093750480937404C596C8CFE091780435
:10359000F091790481E080830E94D7187FCF1F9338
:1035A0001FB781E895E09F938F931F920E9434107C
:1035B000F89411B812B88FEF80937E0080917C0050
:1035C0008F7180937C0080917C00807E80937C0052
:1035D00087E080937A0080917B00887F80937B00D6
:1035E00080917A00886C80937A001FBF78940F9046
:1035F0000F900F9080E995E09F938F931F920E9408
:1036000034100F900F900F901F9108951F920F92FA
:103610000FB60F9211242F933F938F939F93809116
:103620007B04282F33278F5F2330310509F441C0F5
:103630002430310544F52130310509F46CC02230C5
:1036400031050CF44EC080937B04809178009091FA
:1036500079009093A9068093A80683E080937A046A
:1036600080917C00807E90917A04892B80937C00ED
:1036700080917B04882309F46FC080917A00886C64
:1036800080937A0069C025303105C9F125303105B4
:10369000E4F02630310509F44AC02730310509F439
:1036A00052C010927A0410927B0481E08093C00192
:1036B000D7CF80937B04809178009091790090938C
:1036C000AB068093AA0684E0C9CF80937B048091E7
:1036D0007800909179009093B1068093B00685E0D0
:1036E000BDCF232BF1F680937B04809178009091DD
:1036F00079009093B5068093B40681E0AFCF8093B4
:103700007B0480917800909179009093A706809334
:10371000A60686E0A3CF80937B04809178009091E9
:1037200079009093B3068093B20682E097CF80939E
:103730007B0480917800909179009093AD068093FE
:10374000AC0687E08BCF80917800909179009093C0
:10375000AF068093AE06A5CF9F918F913F912F9199
:103760000F900FBE0F901F90189583E995E09F93DF
:103770008F931F920E943410469A3E9882E390E005
:103780000E94491390937D0480937C040F900F90C6
:103790000F9085EA95E09F938F931F920E943410BB
:1037A0000F900F900F900895CF93C0E080917C040C
:1037B00090917D040E945213882301F1369B0BC027
:1037C000C0937E0482E390E00E94491390937D04AD
:1037D00080937C0413C080917E048F5F80937E046D
:1037E000813051F08A3041F080917E048A3051F767
:1037F00087E080937E04E6CFC1E0F6CF8C2F992737
:10380000CF910895CF92DF92EF92FF920F931F9383
:10381000CF93DF938C016A017B0180E090E040E070
:1038200050E060E070E04C155D056E057F05D8F452
:10383000382F2227E92FFF27D8018D918D01992755
:10384000E827F927EE0FFF1FE855FA4F8081918195
:10385000822793274F5F5F4F6F4F7F4F4C155D055A
:103860006E057F0528F3DF91CF911F910F91FF9097
:10387000EF90DF90CF9008952C9A089584B1806BDB
:1038800084B926980E943C1C82E58CBD8DB5816070
:103890008DBD2A9A229808950E943C1C1CBC1DBC18
:1038A00008958FEF8EBD0DB407FEFDCF8EB599271D
:1038B00008958EBD0DB407FEFDCF08952C98089590
:1038C000EF92FF920F931F93CF93DF93EC017A0156
:1038D0008B0140E0542FE114F1040105110509F1B9
:1038E00069E0FE01E50FF11DE081F7E0440F2E2FA6
:1038F000332720783070842F99278078907028178C
:10390000390709F04627EE0FF150F7FFEFCF5F5F61
:10391000852F9927AA27BB278E159F05A007B107DA
:1039200000F3842F9927880F991F482F4160842F17
:103930009927DF91CF911F910F91FF90EF900895FC
:103940000F931F93CF93DF938C010E945E1CC801DD
:103950000E944913EC010E94511C082FCE010E94C5
:103960005213882311F40F3FB1F7802F9927DF916D
:10397000CF911F910F910895CF92DF92EF92FF9216
:103980000F931F93CF93DF93CDB7DEB726970FB674
:10399000F894DEBF0FBECDBF9A01AB01EE24FF2429
:1039A00080648983852F9927AA27BB278A834B8325
:1039B0003C832D8345E050E060E070E0CE0101964D
:1039C0000E94601C8E830E943C1C8FEF0E94591C39
:1039D0000E945E1C84EF91E00E94A01C8E010F5F8C
:1039E0001F4F36E0C32ED12CCC0EDD1EF801819185
:1039F0008F010E94591C8AE090E00197F1F7C016F0
:103A0000D106A0F70E94511C282FC7010894E11C81
:103A1000F11C855F914010F42F3FA1F3822F99276D
:103A200026960FB6F894DEBF0FBECDBFDF91CF91C3
:103A30001F910F91FF90EF90DF90CF900895EF923C
:103A4000FF920F931F93CF93C82F7A018B0140E011
:103A500050E060E070E087E30E94BC1C88232CF0FB
:103A6000B801A7018C2F0E94BC1C9927CF911F91F0
:103A70000F91FF90EF900895AF92BF92CF92DF9297
:103A8000EF92FF920F931F93CF93DF93590167013A
:103A900078010E94BC1C982F8823C9F024E0892F4C
:103AA00099279F938F93C22FDD27DF93CF9388EAC7
:103AB00097E09F938F931F920E9434108DB79EB70B
:103AC00007960FB6F8949EBF0FBE8DBF26C00E940A
:103AD000511C982F807FF9F09E3FC9F7C0E0D0E0DD
:103AE000C114D104E104F10479F085010E94511C54
:103AF000F80181938F012196CE01AA27BB278C154F
:103B00009D05AE05BF0590F30E94511C0E94511CFB
:103B1000C0E0D0E002C02AE0C2CFCE01DF91CF9159
:103B20001F910F91FF90EF90DF90CF90BF90AF90DB
:103B30000895AF92BF92CF92DF92EF92FF920F93D0
:103B40001F93CF93DF93CDB7DEB726970FB6F894C8
:103B5000DEBF0FBECDBF6C01DC018C9199279F9316
:103B60008F938AED97E09F938F931F920E9434105A
:103B7000F601818192819A8389831B820F900F9035
:103B80000F900F900F908E010F5F1F4F1F930F9399
:103B900084EF97E09F938F931F920E94341083E0ED
:103BA00090E0C80ED91E85E0D801F60101900D9273
:103BB0008A95E1F78DEF9FEFC80ED91E1E820F90F8
:103BC0000F900F900F900F901F930F938BE098E042
:103BD0009F938F931F920E9434100F900F900F901D
:103BE0000F900F90F601808599278F7090709F93AA
:103BF0008F93808582958F7099279F938F9380E212
:103C000098E09F938F931F920E9434108DB79EB7B8
:103C100007960FB6F8949EBF0FBE8DBF88E398E05D
:103C20009F938F931F920E9434100F900F900F90CC
:103C3000F7E4AF2EF8E0BF2EE9E0EE2EF12CEC0C0D
:103C4000FD1C03E010E0D7018D917D0199279F9322
:103C50008F93BF92AF921F920E9434100F900F90DB
:103C60000F900F900F900150104017FFECCF8CE495
:103C700098E09F938F931F920E943410F6018685DF
:103C8000482F55274F70507082958F70282F3327FB
:103C90008585992782959295907F9827807F982790
:103CA000282B392B2053384F0F900F900F903F93B4
:103CB0002F935F934F938FE498E09F938F931F927E
:103CC0000E9434108DB79EB707960FB6F8949EBF2A
:103CD0000FBE8DBF26960FB6F894DEBF0FBECDBFC8
:103CE000DF91CF911F910F91FF90EF90DF90CF90D8
:103CF000BF90AF900895EF92FF920F931F93A0E1B2
:103D0000EA2EF12C012D112D9C0140E050E060E0E5
:103D100070E08AE00E943C1D99271F910F91FF904F
:103D2000EF900895EF92FF920F931F93B0E1EB2E67
:103D3000F12C012D112D9C0140E050E060E070E07D
:103D400089E00E943C1D99271F910F91FF90EF90F1
:103D50000895EF92FF920F931F93CF93DF93CDB708
:103D6000DEB726970FB6F894DEBF0FBECDBF1A9907
:103D700082C08AE698E09F938F931F920E9434102E
:103D80000E943E1C0F900F900F9089E798E09F9340
:103D90008F931F920E9434100F900F900F908CE71A
:103DA00098E09F938F931F920E9434101092B60652
:103DB0000E943C1C0F900F900F900EE010E08FEFD0
:103DC0000E94591C0150104017FFF9CF00E010E08D
:103DD00040E050E060E070E080E00E94BC1CF82E03
:103DE0008983C8010F5F1F4F855F914008F053C062
:103DF00081E0F81669F74AEA51E060E070E088E097
:103E00000E94BC1C898387FD25C182FF4DC081E0D3
:103E10008093B70640E050E060E070E08AE30E94E3
:103E2000BC1C898387FD25C182FDF9C08E010E5F10
:103E30001F4FB5E0EB2EF12CEC0EFD1E0E94511C25
:103E4000F80181938F01EE16FF06C0F78B81992749
:103E500080739070C09709F448C08BE099E09F93FD
:103E60008F931F920E94341015E00F900F900F90C7
:103E70000E943C1CADC10E944C1C1092B60611E081
:103E800087EE99E09F938F931F920E9434100F90BA
:103E90000F900F909DC18BE898E09F938F931F9296
:103EA0000E94341012E0E1CF82E08093B7068E01C9
:103EB0000E5F1F4F85E0E82EF12CEC0EFD1E0E94D8
:103EC000511CF80181938F01EE16FF06C0F78D811A
:103ED0008A3A09F092C08C8199278F70907001976F
:103EE00009F498CF88EC98E0BACF80ED97E00E9473
:103EF00049138C0140E050E060E070E089E20E94EC
:103F00001F1D898388230CF493C0C8010E9452139B
:103F1000282F882309F098C0F980F0FCEBCFFF2010
:103F200009F074C040E052E060E070E080E10E947F
:103F3000BC1C082F882309F093C08CEB96E00E94EC
:103F40007B1E182F882309F09AC08CEC96E00E9403
:103F5000921E182F882309F0F7C082EA99E09F93F8
:103F60008F931F930E9434100F900F900F908091A9
:103F7000CC0682958695869583709927009709F4DB
:103F800086C0019709F4F3C01092B8061092B906E2
:103F90001092BA061092BB068091B706992781301D
:103FA000910509F4D9C0029709F40FC18091B806B0
:103FB0009091B906A091BA06B091BB0604E1B695FE
:103FC000A795979587950A95D1F79F938F9382ED43
:103FD00099E09F938F931F920E9434108CEB96E090
:103FE0000E94991D81E08093B6060F900F900F906C
:103FF0000F900F900E943C1CEBC08BEA98E09F93BF
:104000008F931F920E94341014E02FCF8BE499E01D
:104010009F938F932F930E94341013E026CF8BEF42
:1040200098E09F938F931F920E94341016E01DCF4B
:1040300099279F938F9389E299E09F938F931F9283
:104040000E94341014E0D1CF8DE399E09F938F93B9
:104050001F92E1CF99279F938F9389E998E0EDCF45
:1040600087E599E09F938F93FF920E9434101BE0A5
:10407000FCCE99279F938F9388EE98E0DECF8AE756
:1040800099E09F938F93FF920E943410EECE30916F
:10409000D1063F708091D206482F55276627772793
:1040A0004370507060707070AAE0440F551F661F17
:1040B000771FAA95D1F78091D3069927AA27BB2706
:1040C000880F991FAA1FBB1F880F991FAA1FBB1F0C
:1040D000482B592B6A2B7B2B8091D4068295869591
:1040E000869583709927AA27BB27482B592B6A2BC3
:1040F0007B2B2091D5062370220F8091D60699271D
:10410000880F892F881F990B9195282B4F5F5F4F40
:104110006F4F7F4F822F9927029604C0440F551F7F
:10412000661F771F8A95D2F704C0440F551F661F7C
:10413000771F3A95D2F74093B8065093B90660932B
:10414000BA067093BB0628CF8FE899E09F938F93B0
:104150000F930E94341089CE87EA99E09F938F9342
:104160001F920E9434100F900F900F901FCF8091DC
:10417000D3069927AA27BB278F739070A070B070C1
:10418000BC01552744278091D4069927AA27BB272D
:10419000BA2FA92F982F8827482B592B6A2B7B2BB6
:1041A0008091D5069927AA27BB27482B592B6A2B24
:1041B0007B2B83E1440F551F661F771F8A95D1F72C
:1041C00040505040684F7F4FB6CF88EB99E0C6CF44
:1041D000812F992726960FB6F894DEBF0FBECDBF6C
:1041E000DF91CF911F910F91FF90EF90089588EF8D
:1041F00099E09F938F931F920E9434100E944C1C51
:104200001092B6061092B8061092B9061092BA062D
:104210001092BB061092B7060F900F900F9089E096
:104220009AE09F938F931F920E9434100F900F90EB
:104230000F9080E090E00895CF92DF92EF92FF928E
:104240000F931F93CF93DF93DC01CB018A01EE2400
:10425000FF2429E0880F991FAA1FBB1F2A95D1F7B9
:10426000AC01BD0188E10E94BC1CC82F882309F065
:1042700040C0C3E1D0E00E94511C2197D7FFFBCF83
:1042800040E052E060E070E0C8010E94021C6C0156
:104290008EEF0E94591CE80101501E4F89910E9427
:1042A000591C0C171D07D0F78D2D99270E94591CFA
:1042B0008C2D0E94591C0E94511CC82FC7010894C4
:1042C000E11CF11C855F9140A0F52C2F3327C9011B
:1042D00081719070019779F7C9018F7190708B305F
:1042E000910569F18C30910534F50597D9F01CE002
:1042F00001C014E08C2F99279F938F93C12FDD2746
:10430000DF93CF938CE09AE09F938F931F920E944C
:1043100034108DB79EB707960FB6F8949EBF0FBEA8
:104320008DBF27C080ED97E00E94A01CC82F8F3F53
:1043300041F017E0DFCF4D97D1F619E0DBCF18E061
:10434000D9CF40E050E060E070E08DE00E94BC1CFE
:10435000C82F882341F40E94511CC82F882339F4A8
:10436000C0E0D0E006C014E00E94511CC3CF19E0A9
:10437000FBCFCE01DF91CF911F910F91FF90EF9076
:10438000DF90CF900895EF92FF920F931F93DC017F
:10439000CB019A0159E0880F991FAA1FBB1F5A959C
:1043A000D1F7E12C42E0F42E012D112DAC01BD011D
:1043B00081E10E943C1D99271F910F91FF90EF9082
:1043C0000895FC01892B19F08185882329F420E0C8
:1043D00030E040E050E063C0808191818C5B974089
:1043E0009C0144275527A9E1220F331F441F551F65
:1043F000AA95D1F782819927AA27BB278F70907041
:10440000A070B07075E1880F991FAA1FBB1F7A9525
:10441000D1F7282B392B4A2B5B2B83819927AA278D
:10442000BB278F719070A070B070DC01992788272E
:10443000282B392B4A2B5B2B84819927AA27BB2752
:104440008F719070A070B0707BE0880F991FAA1FC9
:10445000BB1F7A95D1F7282B392B4A2B5B2B8581F3
:104460009927AA27BB278F739070A070B07065E062
:10447000880F991FAA1FBB1F6A95D1F7282B392BCC
:104480004A2B5B2B868186959927AA27BB278F719C
:104490009070A070B070282B392B4A2B5B2BCA016F
:1044A000B9010895A0E0B0E060E0AD019A012D509F
:1044B000394FF901E15EFD4F8081882331F06F5F54
:1044C000405E5D4F633090F303C0D90181E080838B
:1044D000CD010895009771F020E0E3EFF6E0E817D2
:1044E000F90749F02F5FE05EFD4F2330C0F380E015
:1044F00090E008950895E15EFD4F1082EF51F24083
:1045000010821182128213821482158216821782FF
:1045100010861286118613861486158616861786CF
:10452000108A118A128A138AE55EFD4F1082118269
:1045300012821382EB51F240148A158A168A178A66
:10454000118E108E128E81E090E00895CF93DF934C
:10455000DC01EB0140E050E030E08C918F3239F427
:1045600042C08F3251F03F5F4115510559F4FD01B2
:10457000E30FF11D80818823A1F7AF013F5F411553
:104580005105A9F31B8680E2FE012AE081932150A8
:1045900027FFFCCF30E0232F8C918F3279F1E32F6E
:1045A000FF27CF018A0F9B1F84179507D0F42B306C
:1045B00038F5EA0FFB1F90819E32D9F0892F815682
:1045C0008A3198F4FE01E20FF11D905290833F5F13
:1045D0002F5FE32FFF27CF018A0F9B1F84179507BB
:1045E00030F3CA010FC031E0C2CFFE01E20FF11D6E
:1045F000EDCF293028F43F5F28E0D1CF31E0CFCF95
:1046000080E090E0DF91CF9108959C018091DC06DD
:10461000882329F420E030E040E050E021C022303F
:10462000310510F422E030E0225030408091DD0668
:104630009927289FA001299F500D389F500D1124C4
:10464000CA019C01442755278091EB069091EC0606
:10465000A091ED06B091EE06280F391F4A1F5B1F8F
:10466000CA01B9010895CF93DF93FC01EB0180915A
:10467000DC06882319F480E090E019C08091EB06F5
:104680009091EC06A091ED06B091EE06C81BD90BF7
:10469000EA0BFB0B8091DD06282F33274427552793
:1046A000BE01CF010E94C042DA01C9010296DF912A
:1046B000CF9108958091DC06992708955F926F92BB
:1046C0007F928F929F92AF92BF92CF92DF92EF92A2
:1046D000FF920F931F93CF93DF93CDB7DEB7C050F8
:1046E000D2400FB6F894DEBF0FBECDBF9C0166244A
:1046F000772443018091DC06882309F47FC0442796
:104700005527220F331F441F551FDA01C90169E0E5
:10471000B695A795979587956A95D1F7E090E306AA
:10472000F090E4060091E5061091E606E80EF91E09
:104730000A1F1B1F9FEFA92E91E0B92EC12CD12C6F
:10474000A222B322C422D5223BC081E0582E11827E
:10475000108244275527220F331F441F551FDA01AB
:10476000C90119E0B695A795979587951A95D1F740
:10477000E090E306F090E4060091E5061091E6066D
:10478000E80EF91E0A1F1B1FBEEFAB2EB1E0BB2EB9
:10479000C12CD12CA222B322C422D522E614F704C4
:1047A0000805190511F4552049F4AE014F5F5F4F1C
:1047B000C401B3010E941C21882301F5552009F191
:1047C000E614F7040805190559F037014801AE0150
:1047D0004F5F5F4FC801B7010E94C321882371F466
:1047E000FE013196EA0DFB1D20813181C90102973E
:1047F0008E5E9F4F08F4A9CF5524A9CF80E090E0AA
:1048000002C081E090E0C050DE4F0FB6F894DEBFEA
:104810000FBECDBFDF91CF911F910F91FF90EF9011
:10482000DF90CF90BF90AF909F908F907F906F90D0
:104830005F900895CF92DF92EF92FF920F931F93B4
:10484000CF93DF93EC01892B09F474C08091DC06CF
:10485000882309F46FC08B8599278136910521F053
:104860008737910509F066C089859A85892B09F0FB
:1048700049C0ABE1EA2EF12CEC0EFD1EFBE1CF2E80
:10488000F2E0DF2ECC0EDD1E8C899D89AE89BF89BA
:10489000F60180839183A283B383A701BC01CD017C
:1048A0000E94C321882309F043C0088D198D000F91
:1048B000111F02951295107F1027007F10270E0DF3
:1048C0001F1D8C859D85AE85BF85F801848F958FD2
:1048D000A68FB78F8CE996E00E94E121DC01CB0125
:1048E000F801868B978BA08FB18FA701F6016081AD
:1048F0007181828193810E941C218823C9F480E008
:1049000090E01AC01BE1E12EF12CEC0EFD1EBBE184
:10491000CB2EB2E0DB2ECC0EDD1EA701F6016081AE
:104920007181828193810E941C21882309F4ACCF7C
:104930000E94BA248FEF9FEFDF91CF911F910F91CB
:10494000FF90EF90DF90CF9008950F931F93CF9338
:10495000DF93EC010FEF1FEF009731F00E941A2454
:104960008C01CE010E946A22C801DF91CF911F9174
:104970000F910895EF92FF921F93CF93DF93EE2450
:10498000FF24C3EFD6E012E0C15EDD4F8881CF5136
:10499000D240813031F01150C05EDD4F17FFF4CFAF
:1049A00006C0CE010E94A524E80EF91EF4CF0E9495
:1049B000F7201092DC068E2D9927DF91CF911F9161
:1049C000FF90EF9008952F923F924F925F926F92D7
:1049D0007F928F929F92AF92BF92CF92DF92EF928F
:1049E000FF920F931F93CF93DF93CDB7DEB724973A
:1049F0000FB6F894DEBF0FBECDBFAC011A8219828C
:104A00008091DC06882309F488C04115510509F41A
:104A100084C08824992454019BE1292E92E0392EE8
:104A2000240E351E8A01055E1F4F24013501809139
:104A3000E3069091E406A091E506B091E606880DA4
:104A4000991DAA1DBB1DF10180839183A283B383AD
:104A5000A801BC01CD010E94C321882309F05BC0DD
:104A60001C821B8273016201F694E794D794C79469
:104A700009C0AB81BC811196BC83AB83AF3FB1054C
:104A800009F058F5EB81FC81EE0FFF1FE00FF11FDD
:104A900080819181892B69F78FEF9FEF91838083CC
:104AA000A801D1016D917D918D919C910E941C2155
:104AB000882389F5EB81FC81EC0DFD1DFA83E983E8
:104AC00080E091E09C838B83AB81BC811196BC8399
:104AD000AB83AF3FB105B1F2A8F20894811C911CE1
:104AE000A11CB11C80E092E0A0E0B0E0480E591E8D
:104AF0006A1E7B1E8091E1069091E206AA27BB27E1
:104B000088169906AA06BB0640F4A981BA81AB2B88
:104B100009F48DCF02C00E94BA2489819A8124961B
:104B20000FB6F894DEBF0FBECDBFDF91CF911F91BE
:104B30000F91FF90EF90DF90CF90BF90AF909F903C
:104B40008F907F906F905F904F903F902F9008953F
:104B5000AF92BF92CF92DF92EF92FF920F931F938B
:104B6000CF93DF938C01EE24FF248091DC06882311
:104B700009F489C00115110509F485C08091EB067F
:104B80009091EC06A091ED06B091EE06F80124811B
:104B9000358146815781281739074A075B0708F492
:104BA00072C08091EF069091F006A091F106B0914D
:104BB000F20682179307A407B50708F464C0CA0178
:104BC000B9010E9433237C01C701AA27BB27880FA4
:104BD000991FAA1FBB1F9C01AD0169E0569547951F
:104BE000379527956A95D1F7C091E306D091E406F1
:104BF000E091E506F091E606C20FD31FE41FF51F12
:104C00002FEFA22E21E0B22EC12CD12CA822B92246
:104C1000CA22DB229801255E3D4FD9014D915D915D
:104C20006D917C9113974C175D076E077F0771F0AC
:104C3000CD93DD93ED93FC931397C8014B96AC0194
:104C4000BE01CF010E94C321882369F4F801EA0D57
:104C5000FB1DE38CF48CB8EFEB16BFEFFB0630F0D6
:104C6000EE24FF2410C00E94BA240DC0C7010E9488
:104C70000523DC01CB01F80184839583A683B783E8
:104C8000108612861186C701DF91CF911F910F9177
:104C9000FF90EF90DF90CF90BF90AF9008952F924C
:104CA0003F924F925F926F927F928F929F92AF92BC
:104CB000BF92CF92DF92EF92FF920F931F93CF9309
:104CC000DF93CDB7DEB72E970FB6F894DEBF0FBED9
:104CD000CDBF9A8389836B834C8319011A86198609
:104CE00000E08091DC06882309F4B0C0232B09F48E
:104CF000ADC029813A81232B09F4A8C0D1011D92AE
:104D00001D921D921C921397F101C488D588E688E4
:104D1000F788C114D104E104F10409F09AC080912C
:104D2000DF069091E006880F991F82959295907FFB
:104D30009827807F9827892F992786959C0144275B
:104D400055272D833E834F8358878091E7069091A6
:104D5000E806A091E906B091EA0680839183A283D8
:104D6000B383F10180819181A281B3810097A10574
:104D7000B10509F40FC19101255E3D4F3C872B879A
:104D80001BE1812E912C820C931C9C01AD01F10141
:104D900084839583A683B783108612861186442464
:104DA0005524320159016A01A40CB51CC61CD71C3C
:104DB000AB85BC85AD92BD92CD92DC921397A401D8
:104DC000C601B5010E94C3218823F1F5EE24FF241A
:104DD000A701440F551F42955295507F5427407F9D
:104DE0005427FA01E80DF91DFE87ED872081822FF7
:104DF0009927009751F0853E910539F08385FC8114
:104E00008F233B81831709F457C00894E11CF11CE0
:104E1000F0E1EF16F104E0F20894411C511C611C12
:104E2000711C2D813E814F815885421653066406C0
:104E3000750608F0E7C0002309F0E4C0F101248101
:104E4000358146815781AECF0E94BA2480E090E040
:104E50000FC18091E7069091E806A091E906B09114
:104E6000EA06C816D906EA06FB0608F470C0809167
:104E7000EB069091EC06A091ED06B091EE06C816F7
:104E8000D906EA06FB0608F06AC08091DF06909119
:104E9000E006880F991F82959295907F9827807FD2
:104EA0009827892F992786959C01442755272D837C
:104EB0003E834F83588755CF30E0A981BA818C91CA
:104EC000281709F0A2CF3F5F3B3078F4632F772794
:104ED000AD85BE85A60FB71FE981FA816E0F7F1FD2
:104EE0009C91DB018C91981771F33A3008F48DCFC7
:104EF0008A01080D191DF8018385F101828FF801DF
:104F0000828D938D0E940523DC01CB01F10180830A
:104F10009183A283B38384839583A683B78310860A
:104F200012861186A48AB58AC68AD78AF18EE08E47
:104F3000F801848D958DA68DB78DF10184879587B5
:104F4000A687B78701E0E0E1EE2EF12C5ECF8091DD
:104F5000EB069091EC06A091ED06B091EE06C81616
:104F6000D906EA06FB0608F471CF8091EF0690910E
:104F7000F006A091F106B091F2068C159D05AE05E4
:104F8000BF0508F463CF8091DD06282F332744271F
:104F900055278DCF9101255E3D4F3C872B87D90149
:104FA000CD92DD92ED92FC9213979BE1892E912C8C
:104FB000820C931CA401C701B6010E94C32188235F
:104FC00009F042CFF101A08DB18DAA0FBB1FA295B0
:104FD000B295B07FBA27A07FBA27A80DB91D8C91D2
:104FE0009927009709F432CF853E910509F42ECF19
:104FF000FD01838599279C012071307084FD2BC0B1
:10500000C90136C0002391F48091EB069091EC0623
:10501000A091ED06B091EE06F10124813581468123
:105020005781281739074A075B0760F429853A85B5
:10503000232B71F0002361F4F10124813581468135
:105040005781ADCEC1010E94A8259A878987EECFEE
:10505000802F99270DC0FD01828D938D0E9405231D
:10506000DC01CB01F10180839183A283B3838DCED8
:105070002E960FB6F894DEBF0FBECDBFDF91CF9155
:105080001F910F91FF90EF90DF90CF90BF90AF9066
:105090009F908F907F906F905F904F903F902F9058
:1050A0000895BF92CF92DF92EF92FF920F931F93DA
:1050B000CF93DF93CDB7DEB72C970FB6F894DEBF52
:1050C0000FBECDBFFC01B62EC42E790100E010E06A
:1050D000DD24892B39F02115310521F08091DC0682
:1050E000882319F480E090E033C0DF01F901148ACD
:1050F000158A168A178A118F008F8C918823C1F424
:105100008D2D992725C06B2D4C2D9701CE01019631
:105110000E944F268823A1F3F8018081882311F48F
:1051200061E0D62ED8018C91882351F3DD2041F720
:10513000BE016F5F7F4FCD010E94A6228C010097B8
:10514000F9F2FC0180818823F1F260E148E1DDCFD2
:105150002C960FB6F894DEBF0FBECDBFDF91CF9176
:105160001F910F91FF90EF90DF90CF90BF90089527
:10517000AF92BF92CF92DF92EF92FF920F931F9365
:10518000CF93DF93EC01EE24FF248701E1E0CE2EE4
:10519000D12C8091DC06882309F45DC0209709F4A6
:1051A0005AC02115310541F02230310509F465C09E
:1051B000E888F9880A891B89E40EF51E061F171F67
:1051C00017FD4CC08C859D85AE85BF858E159F05CE
:1051D000A007B1070CF442C088819981AA81BB81E4
:1051E0008C839D83AE83BF8318861A861986188A9E
:1051F000198A1A8A1B8A80E090E0A0E0B0E08E1540
:105200009F05A007B10770F5A12C72E0B72E12C060
:105210001A86198688858F5F88879091DD068917A1
:1052200088F588899989AA89BB898E159F05A00769
:10523000B107C0F40196A11DB11D888B998BAA8B73
:10524000BB8B89859A85019622E08030920700F712
:105250009A878987E6CF80E090E021C08889998984
:10526000AA89BB898E159F05A007B10711F0C60159
:1052700016C0CC24DD24C60112C0EC84FD840E854A
:105280001F859ACFCE010E94A825892B11F0188680
:10529000C8CF888581508887BA86A986C2CFDF911A
:1052A000CF911F910F91FF90EF90DF90CF90BF9023
:1052B000AF9008956F927F928F929F92AF92BF921C
:1052C000CF92DF92EF92FF920F931F93CF93DF93D2
:1052D0008C01EE24FF248091DC06882349F001151F
:1052E000110531F0C8010E94E3247C01892B11F4DF
:1052F000C7017FC022E030E040E050E060E070E0B5
:10530000C8010E94B828F80164817581868197815F
:105310000E943323AA27BB27880F991FAA1FBB1FF0
:105320009C01AD0169E056954795379527956A959B
:10533000D1F7C091E306D091E406E091E506F09143
:10534000E606C20FD31FE41FF51F2FEF622E21E0E8
:10535000722E812C912C682279228A229B22BBE119
:10536000AB2EB2E0BB2EA00EB11ED5012D913D910A
:105370004D915C9113972C173D074E075F0779F10C
:10538000CD93DD93ED93FC931397ABE1CA2ED12C13
:10539000C00ED11EA601BE01CF010E94C3218823E9
:1053A00021F5F801E60DF71DF48EE38EA601F50157
:1053B00060817181828193810E941C21C82F882382
:1053C000A1F4C7010E940523DC01CB01F80184830D
:1053D0009583A683B783C0871286118689CFFBE1A8
:1053E000CF2ED12CC00ED11EDCCF0E94BA2480E07B
:1053F00090E0DF91CF911F910F91FF90EF90DF90A0
:10540000CF90BF90AF909F908F907F906F900895B6
:105410009F92AF92BF92CF92DF92EF92FF920F9343
:105420001F93CF93DF93EC01A1E09A2E8091DC06CD
:10543000882309F452C0209709F44FC0EE24FF24BA
:105440008701FE01EE0DFF1D138E0894E11CF11C77
:10545000011D111D80E0E81682E0F80680E00807D3
:1054600080E0180770F3EE24FF2487018091DD06A9
:105470008823B1F1FBE1AF2EF2E0BF2EAC0EBD1ED2
:10548000EBE1CE2ED12CCC0EDD1E0FC00894E11C1A
:10549000F11C011D111D8091DD069927AA27BB274C
:1054A000E816F9060A071B07D8F48C819D81AE81A6
:1054B000BF818E0D9F1DA01FB11FF50180839183B9
:1054C000A283B383A601BC01CD010E941C218823C5
:1054D000E9F20E94BA249924D9CF80E090E002C07A
:1054E000892D9927DF91CF911F910F91FF90EF9018
:1054F000DF90CF90BF90AF909F9008952F923F92F2
:105500004F925F926F927F928F929F92AF92BF92D3
:10551000CF92DF92EF92FF920F931F93CF93DF937F
:10552000CDB7DEB761970FB6F894DEBF0FBECDBF23
:105530009A838983362E8A01CC24DD24DC86CB86AF
:10554000DE86CD8622248091DC06882309F480C083
:105550004115510509F47CC029813A81232B09F4B6
:1055600077C0DA011D921D921D921C921397FA01C9
:10557000A488B588C688D788A114B104C104D10411
:1055800009F069C08091DF069091E006880F991FAD
:1055900082959295907F9827807F9827892F9927C9
:1055A00086959C01442755272F83388749875A873A
:1055B0004D855E855C874B878091E7069091E80674
:1055C000A091E906B091EA0680839183A283B38318
:1055D000F80180819181A281B3810097A105B10575
:1055E00009F07BC0055E1D4FD801AD92BD92CD92F2
:1055F000DC9213970B511240FBE1EF2EF12CE00EE1
:10560000F11EA701C601B5010E94C3218823F1F450
:10561000F801A08DB18DAA0FBB1FA295B295B07FE6
:10562000BA27A07FBA27AE0DBF1D8C91992700978E
:1056300079F0853E910561F0FD01838599279C01F4
:105640002071307084FD3AC0C901B1C10E94BA24F2
:1056500080E090E0ACC18091E7069091E806A091CF
:10566000E906B091EA06A816B906CA06DB0608F4F0
:1056700054C18091EB069091EC06A091ED06B0919B
:10568000EE06A816B906CA06DB0608F04EC18091E0
:10569000DF069091E006880F991F82959295907F82
:1056A0009827807F9827892F992786959C014427E2
:1056B00055272F83388749875A878ACFFD01A28DC6
:1056C000B38DBC87AB87CD010E940523DC01CB01E4
:1056D000F80180839183A283B383C8010E94E324ED
:1056E0003C01892B09F416C1D8012D913D914D91B2
:1056F0005C91F801248335834683578310867BE1D0
:10570000472E72E0572E400E511E6BE1E62EF12C13
:10571000E00EF11E1B821C821D821E828B809C80EB
:10572000AD80BE80820E931EA41EB51ED2018D9246
:105730009D92AD92BC921397A701C501B4010E943E
:10574000C321882309F082CFCC24DD240AC0853E02
:10575000B1F00894C11CD11CB0E1CB16D10408F003
:1057600068C0F601EE0FFF1FE295F295F07FFE276D
:10577000E07FFE27EE0DFF1D8081882341F7F98B26
:10578000E88BDF0129813A819AE0F90181919F013B
:105790008D93915097FFF9CFE889F9893386738EFD
:1057A000628E8CE996E00E94E121DC01CB01E88960
:1057B000F989868B978BA08FB18F148E158E168EDC
:1057C000178EA701D2016D917D918D919C910E94C0
:1057D0001C218F87882309F09BC0C3010E940523E9
:1057E000DC01CB01F80180839183A283B38384839E
:1057F0009583A683B7832F85208712861186328EE4
:105800001486158616861786848A958AA68AB78A8C
:10581000D18EC08E34FC2CC081E0282EB0E1CB2E7E
:10582000D12C0894C11CD11CB0E1CB16D10408F4D2
:1058300098CF2B813C814D815E812F5F3F4F4F4F31
:105840005F4F2B833C834D835E838F819885A98531
:10585000BA85281739074A075B0708F081C022205C
:1058600009F07EC0F801248135814681578156CFE9
:10587000C8010E94082AF80180819181A281B38128
:10588000F20180839183A283B383A701BC01CD0180
:105890000E94C3218823E1F52EE2F801238F20E244
:1058A000F701319699E02193915097FFFCCF80E169
:1058B000F7018387738E628E168A178A108E118E77
:1058C000148E158E168E178E3EE230A331A3822FD2
:1058D000B29698E08193915097FFFCCF80E1F70159
:1058E00083A72B853C8533AF22AF16AA17AA10AE2B
:1058F00011AE14AE15AE16AE17AEA701D2016D9162
:105900007D918D919C910E941C21882309F484CF64
:105910000E94BA24822D99274AC08091EB0690916B
:10592000EC06A091ED06B091EE06A816B906CA06DF
:10593000DB0608F48DCE8091EF069091F006A091E1
:10594000F106B091F2068A159B05AC05BD0508F479
:105950007FCE8091DD06282F332744275527A9CEF7
:105960002220B9F48091EB069091EC06A091ED060F
:10597000B091EE06F80124813581468157812817C0
:1059800039074A075B0728F0C8010E94A8259E87AF
:105990008D872D853E85232B09F4BCCF222009F06D
:1059A000B9CFF8012481358146815781B3CE619604
:1059B0000FB6F894DEBF0FBECDBFDF91CF911F9120
:1059C0000F91FF90EF90DF90CF90BF90AF909F909E
:1059D0008F907F906F905F904F903F902F900895A1
:1059E000BF92CF92DF92EF92FF920F931F93CF93CC
:1059F000DF93CDB7DEB72C970FB6F894DEBF0FBE9E
:105A0000CDBF9C01B62E7A0100E010E0CC24892B9A
:105A100039F04115510521F08091DC06882319F4F5
:105A200080E090E041C0D901FA01148A158A168AF3
:105A3000178A118F008F8C91882331F58C2D99272F
:105A400033C0D62E970148E16D2DCE0101960E94FC
:105A50004F26882399F4F8018081882309F4DB2CF0
:105A6000A7016D2DCE0101960E947E2A882331F375
:105A7000F8018081882311F441E0C42ED8018C9173
:105A80008823E1F2CC20D1F6BE016F5F7F4FCD01BC
:105A90000E94A6228C01009789F2FC016081662396
:105AA00081F250E1D52ECECF2C960FB6F894DEBF02
:105AB0000FBECDBFDF91CF911F910F91FF90EF905F
:105AC000DF90CF90BF900895FF920F931F93CF93D5
:105AD000DF938C01F62EC0E0D0E08091DC068823B5
:105AE00009F49BC00115110509F497C00E945222C8
:105AF000EC01892B09F491C0188219821A821B8249
:105B00001C821D821E821F8218861A861986FB86B9
:105B10001C861D861E861F86188A198A1A8A1B8A69
:105B2000C55EDD4F188219821A821B82CB51D2408A
:105B30001C8A1D8A1E8A1F8A198E188E1A8E9E0133
:105B400048E16885C8010E945128882309F441C0B2
:105B50006F2D772767FD70956237710509F45AC07C
:105B6000633771050CF445C067377105E1F58A8D1F
:105B700099278C010170107080FD35C06881798192
:105B80008A819B810E9433230E945E23CE010E9462
:105B9000E3240E940523DC01CB0188839983AA8337
:105BA000BB838C839D83AE83BF8318861A87098746
:105BB0001C861D861E861F86188A198A1A8A1B8AC9
:105BC000980140E050E060E070E0CE010E94B8280B
:105BD00024C06F2D772767FD70956136710591F0B0
:105BE0006737710579F0CE010E94A524C0E0D0E0AE
:105BF00014C061367105B9F78A8D80FDF4CF22E0BB
:105C000030E0DFCFAE0160E2C8010E94F02C8823B3
:105C100021F4E9CF20E030E0D4CFCE01DF91CF9165
:105C20001F910F91FF9008958F929F92AF92BF9214
:105C3000CF92DF92EF92FF920F931F93CF93C0E02A
:105C40008BE39AE09F938F93CF930E943410C0937D
:105C5000DC060F900F900F90E2E1F9E082E01082F5
:105C6000E05EFD4F815087FFFACF0E94A91EC82F2A
:105C7000882309F0A9C04EE057E060E070E080E0C2
:105C800090E00E94C321882309F0EAC08091D008E7
:105C9000843009F4C2C0863009F4BFC08E3009F4E4
:105CA000BCC08824992454018091190790911A0747
:105CB0008050924009F0CBC080911B078093DD0695
:105CC00040911E074093DE06C0901F07D09020072A
:105CD000D092E006C092DF0620912407309125077C
:105CE0003093E2062093E10680911C0790911D07F6
:105CF0007C0100271127E80CF91C0A1D1B1DE092EE
:105D0000E306F092E4060093E5061093E606C90167
:105D1000AA27BB27242F332744275527BC01CD01B1
:105D20000E947A42DC01CB018E0D9F1DA01FB11F86
:105D30008093E7069093E806A093E906B093EA06FD
:105D4000D294C2946FE0C622CD24D622CD249601EF
:105D500044275527280F391F4A1F5B1F2093EB0646
:105D60003093EC064093ED065093EE0680912E079B
:105D700090912F07A0913007B09131070097A105AE
:105D8000B10509F476C0280F391F4A1F5B1F215047
:105D90003040404050402093EF063093F00640934F
:105DA000F1065093F20680914407863421F48091E5
:105DB00045078134B9F088ED9AE09F938F931F9245
:105DC0000E943410C6E008C08CE49AE09F938F9341
:105DD0001F920E943410C1E00F900F900F900E940C
:105DE000BA2450C080914607843529F7809147072F
:105DF000813309F7809148078633E9F681E0809383
:105E0000DC06C0E08BEF9AE09F938F93CF930E94C4
:105E100034100F900F900F9035C08090D408909060
:105E2000D508A090D608B090D7084EE057E0C5013D
:105E3000B4010E94C321882309F436CF85E89AE093
:105E40009F938F931F920E943410C3E0C5CF8CE9BB
:105E50009AE09F938F931F920E943410C4E0BCCFAE
:105E60008EE69AE09F938F93CF930E943410C2E006
:105E7000B3CF8CEB9AE09F938F931F920E943410C4
:105E8000C5E0AACF8C2F9927CF911F910F91FF903A
:105E9000EF90DF90CF90BF90AF909F908F9008953C
:105EA000AF92BF92CF92DF92EF92FF920F931F9328
:105EB000CF93DF93EC017FEFA72EB72E8091DC0606
:105EC000882309F472C0209709F46FC02C853D85A2
:105ED0004E855F85211531054105510509F465C0E1
:105EE000C888D988EA88FB88D701C6010196A11D18
:105EF000B11D82179307A407B50708F056C00C819F
:105F00001D812E813F818885080F111D211D311DA6
:105F1000FE01E55EFD4F80819181A281B3818017F2
:105F20009107A207B30789F000831183228333838B
:105F3000CE014B96AC01C901B8010E94C321882350
:105F400051F5C888D988EA88FB8889859A85FE0139
:105F5000E80FF91F238DA22EBB240894C11CD11C6D
:105F6000E11CF11CC88AD98AEA8AFB8A019622E0E0
:105F700080309207C0F01A86198688858F5F8887DF
:105F80009091DD06891788F0CE010E94A825892B03
:105F900029F018860AC00E94BA2407C0888581505B
:105FA000888780E092E09A878987C501DF91CF9149
:105FB0001F910F91FF90EF90DF90CF90BF90AF9027
:105FC00008958F929F92AF92BF92DF92EF92FF92CD
:105FD0000F931F93CF93DF93D82E8B018091DC0614
:105FE000882309F46FC06115710509F46BC0FB01CA
:105FF000208931894289538984859585A685B7850D
:10600000281739074A075B0708F050C0F801848059
:106010009580A680B7808085880E911CA11CB11C3C
:10602000EBE1EE2EE2E0FE2EE00EF11EF7018081A4
:106030009181A281B38188159905AA05BB0571F0EC
:1060400080829182A282B382C8014B96AC01C501C5
:10605000B4010E94C321882309F074C0F80161854E
:106060007285E60FF71FD38EF80184859585A68586
:10607000B785208931894289538982179307A407FC
:10608000B50709F441C02F5F3F4F4F4F5F4FF801F5
:10609000208B318B428B538BCB010196928781876A
:1060A0008050924090F480E090E050C081859285CD
:1060B0008050924008F4AACFCB010E945A29892B24
:1060C00009F0A4CF8FEF9FEF41C0C8014B96AC0100
:1060D000F70160817181828193810E941C21C82F08
:1060E000882381F5F8011286118680858F5F80876D
:1060F0009091DD068917B8F2C8010E94A825892B66
:1061000081F0F801C087CFCF2F5F3F4F4F4F5F4FD8
:10611000248735874687578721503040404050407C
:10612000B2CFC8010E945A29892B09F0BCCFF801CF
:1061300080858150808780E092E0928781878FEF11
:106140009FEF04C00E94BA248FEF9FEFDF91CF91A1
:106150001F910F91FF90EF90DF90BF90AF909F90B5
:106160008F9008952F923F925F926F927F928F92BD
:106170009F92AF92BF92CF92DF92EF92FF920F93D6
:106180001F93CF93DF93FC015A016B013801490142
:106190001701EE24FF248701A1E05A2E8091DC062E
:1061A0008823A9F12114310491F1309781F1EF0195
:1061B000E614F7040805190538F5A114B104C10463
:1061C000D104A1F0552091F0C1010E94502F2FEF72
:1061D0008F3F920709F189930894A108B108C1087B
:1061E000D108A114B104C104D10461F7552029F0EC
:1061F0000894E11CF11C011D111DE614F7040805AB
:10620000190510F45520C9F6C801B70107C060E0B0
:1062100070E080E090E002C05524CFCFDF91CF91B5
:106220001F910F91FF90EF90DF90CF90BF90AF90B4
:106230009F908F907F906F905F903F902F900895E8
:106240002F923F925F926F927F928F929F92AF9226
:10625000BF92CF92DF92EF92FF920F931F93CF9353
:10626000DF93FC015A016B01380149011701EE244B
:10627000FF248701B1E05B2E8091DC068823A9F121
:106280002114310491F1309781F1EF01E614F70404
:106290000805190538F5A114B104C104D104A1F011
:1062A000552091F0B10188810E94E12F8F5F9F4FAF
:1062B00009F121960894A108B108C108D108A114D8
:1062C000B104C104D10461F7552029F00894E11C00
:1062D000F11C011D111DE614F7040805190510F441
:1062E0005520C9F6C801B70107C060E070E080E042
:1062F00090E002C05524CFCFDF91CF911F910F9135
:10630000FF90EF90DF90CF90BF90AF909F908F90D5
:106310007F906F905F903F902F900895FF920F9322
:106320001F93CF93DF93EC018B01FF2420E030E03B
:106330008091DC068823F1F0672BE1F02097D1F003
:1063400088818823A9F0D901AC0FBD1FB8018C91B9
:106350000E94E12F9C01F394AF2DBB27FE01EA0FB1
:10636000FB1F8081882321F08FEF2F3F380761F7D3
:10637000C90102C080E090E0DF91CF911F910F91A1
:10638000FF900895CF92DF92EF92FF920F931F93A9
:10639000CF93DF937C016A018091DC06882321F191
:1063A000452B11F1E114F104F9F016161706E4F487
:1063B0008701EB01C230D1058CF0C6010E94502F3D
:1063C0002FEF8F3F920771F08A30910539F0F80175
:1063D00081938F012197C230D1057CF7F80110829B
:1063E000C70104C0F801108280E090E0DF91CF91F6
:1063F0001F910F91FF90EF90DF90CF900895EF9253
:10640000FF920F931F93CF937C01C0E00E94522212
:106410008C019C0148E16C2FC7010E945128C82FB4
:10642000C8010E946A228C2F9927CF911F910F914A
:10643000FF90EF900895FC0180899189A289B3892A
:106440000196A11DB11D2485358546855785821786
:106450009307A407B50718F480E090E0089581E061
:1064600090E00895CF93DF93FC01EB0190E030972B
:1064700021F1672B11F18485882319F4892F99273D
:106480001EC080819181A281B38188839983AA8370
:10649000BB8384819581A681B7818C839D83AE83E4
:1064A000BF8380859185A285B38588879987AA87D0
:1064B000BB8781E08C87982FE1CF80E090E0DF916F
:1064C000CF910895FC01009781F010821182128211
:1064D0001382148215821682178210861186128604
:1064E0001386148681E090E0089508958091F20368
:1064F00099278130910519F18230910584F0029736
:1065000019F01092F203089580917F049091800415
:106510000E9452138823B9F31092F2030895892B35
:1065200081F780919F039091A00381609093A003D5
:1065300080939F038EE895E00E946232089588EE72
:1065400093E00E9449139093800480937F0480918C
:106550009F039091A0038E7F9093A00380939F034D
:10656000809181049091820401969093820480939B
:1065700081048091D503992783709070892B21F035
:106580008091D403843090F58EE895E00E946232C9
:1065900080919E03823021F082E08093F20308957F
:1065A0008091D30380FD11C0809181049091820479
:1065B00065E070E00E949942892B39F484E690E00E
:1065C0009093BF038093BE03E7CF8091D4038430C0
:1065D00018F7809181049091820465E070E00E9438
:1065E0009942892BC9F68AE090E0EACF6EE875E01F
:1065F00086EC93E00E943232CBCFE1ECF1E021E077
:1066000085899689948B838B21507B9627FFF8CFC1
:1066100008958F929F92AF92BF92CF92DF92EF92A6
:10662000FF920F931F93CF93DF93CDB7DEB762979F
:106630000FB6F894DEBF0FBECDBF7C014B0100E06A
:106640005E010894A11CB11C82E127EF31E0D50165
:10665000F90101900D928A95E1F7E114F10409F432
:1066600040C0672BF1F1F70101900020E9F7319765
:106670001E2F1E19113198F5812F9927AC01B701F2
:10668000C5010E94EC3E102F81ECC82E81E0D82E6F
:1066900076010894E11CF11C40E150E0B701CE0105
:1066A00001960E94F93E892BF9F01F5FABE1B0E043
:1066B000EA0EFB1ECA0EDB1E123070F3BF92AF92C1
:1066C00088E29BE09F938F930F930E9434100F906A
:1066D0000F900F900F900F90802F992738C010E1E6
:1066E000CBCF80E090E033C0C4010E94A53EF7010B
:1066F000938B828B268937898217930708F5F601D9
:10670000618D728D7F936F933F932F939F938F93A0
:10671000BF92AF9282E09BE09F938F931F920E9463
:106720003410F60185899689948B838B8DB79EB73B
:106730000B960FB6F8949EBF0FBE8DBF01E0CCCF75
:10674000608D718D68177907E8F201E0C5CF629618
:106750000FB6F894DEBF0FBECDBFDF91CF911F9172
:106760000F91FF90EF90DF90CF90BF90AF909F90F0
:106770008F9008956F927F928F929F92BF92CF9247
:10678000DF92EF92FF920F931F93CF93DF93CDB7DA
:10679000DEB7A2970FB6F894DEBF0FBECDBF85E47B
:1067A0009BE09F938F931F920E9434100E94FD32B2
:1067B0000E945A23282F0F900F900F90882309F4DE
:1067C00050C089E092E00E94FF31F82E882309F43E
:1067D0004EC062E789E092E00E94642D8C01892B13
:1067E00009F493C0A80160E270E0CE0101960E9416
:1067F000C231892B81F189818A30A1F38D3091F3E7
:10680000803281F38B3371F3833261F3AE014F5DDC
:106810005F4F66E172E0CE0101960E94073F7C0166
:10682000AE014F5D5F4F66E172E080E090E00E9454
:10683000073FBC01E114F104A9F2892B99F2C701C9
:106840000E940933A80160E270E0CE0101960E9427
:10685000C231892B81F6C8010E94A52487E79BE0FD
:1068600050C080EC9BE09F938F932F9356C067E7B7
:1068700089E092E00E94642D8C01892B09F448C0C4
:1068800048E1642E42E0742E4E010894811C911C54
:1068900032ECE32E31E0F32E24E1C22ED12CCE0CCB
:1068A000DF1C91E0B92EF601808191812BE130E06F
:1068B000C20ED31E9F938F93FF92EF927F926F929F
:1068C0009F928F920E94413FB801C4010E948E3175
:1068D0008DB79EB708960FB6F8949EBF0FBE8DBFBA
:1068E000BA94EBE1F0E0EE0EFF1EB7FEDCCFB8018C
:1068F00082E292E00E948E31C8010E94A52481EAC2
:106900009BE09F938F931F9208C089E59BE0F9CF8E
:106910008AE79BE09F938F93FF920E9434100F9021
:106920000F900F90A2960FB6F894DEBF0FBECDBFAA
:10693000DF91CF911F910F91FF90EF90DF90CF905B
:10694000BF909F908F907F906F900895382FDB01BC
:1069500090E0292FE1ECF1E08081831729F02F5F8F
:106960007B962230C8F305C0838994898D939C93CC
:1069700091E0892F992708950F931F938091A50681
:10698000882309F45CC08091A8049091A904209107
:106990009C0630919D068217930709F441C05091DF
:1069A0009E0640919F063093A9042093A80450931B
:1069B000AA044093AB0481E08093B1041092840454
:1069C0001092830480918304909184049F938F9309
:1069D000842F99279F938F93852F99279F938F9328
:1069E0003F932F9389E292E09F938F9305E814E001
:1069F0001F930F930E94413F8091830490918404E0
:106A000001969093840480938304C8012DB73EB708
:106A1000245F3F4F0FB6F8943EBF0FBE2DBF11C08D
:106A20008091AA0450919E06851709F0BACF8091F3
:106A3000AB0440919F06841709F0B5CFC3CF80E027
:106A400090E01F910F9108950F931F938091A506D9
:106A5000882309F45CC08091D7049091D8042091D8
:106A60009C0630919D068217930709F441C050910E
:106A70009E0640919F063093D8042093D7045093EC
:106A8000D9044093DA0481E08093E0041092B304C7
:106A90001092B2048091B2049091B3049F938F93AB
:106AA000842F99279F938F93852F99279F938F9357
:106AB0003F932F938AE492E09F938F9304EB14E02B
:106AC0001F930F930E94413F8091B2049091B304B1
:106AD00001969093B3048093B204C8012DB73EB7DA
:106AE000245F3F4F0FB6F8943EBF0FBE2DBF11C0BD
:106AF0008091D90450919E06851709F0BACF8091F4
:106B0000DA0440919F06841709F0B5CFC3CF80E027
:106B100090E01F910F910895CF93DF93EC01892BA3
:106B2000D1F48091E104833009F44AC01092E10469
:106B3000D093E304C093E20488EE94E00E945D38B1
:106B4000CE010E9449139093E5048093E404809160
:106B5000E104992719C18091E4049091E5040E9411
:106B60005213882329F49091E104892F99270CC1AD
:106B7000CE010E9449139093E5048093E404809130
:106B80009E03823011F19091E104933071F788EE09
:106B900094E00E94F338282F882309F487C081E508
:106BA0009CE09F938F931F920E94341082E0809309
:106BB000E1040F900F900F90982F892F9927E4C030
:106BC00088EE94E00E94F338B1CF9091E104292F30
:106BD00033272230310509F44CC0233031050CF045
:106BE0005BC02115310509F444C02130310531F075
:106BF0001092E10490E0892F9927C6C00E94BC340E
:106C00009093E3048093E204009721F00E94FF3107
:106C10008823A1F78091E2049091E304009709F49E
:106C200070C068EE74E00E946438282F882309F44D
:106C300078C080E29EE40E9449139093E704809319
:106C4000E60483E08093E1048091E2049091E30400
:106C50009F938F9386ED9BE09F938F931F920E944B
:106C600034100F900F900F900F900F909091E104BF
:106C70007CCF8091F203882309F477CF8091D303EE
:106C800080FF73CF8091D503833009F06ECF81E010
:106C90008093E104982F91CF2330310581F0243087
:106CA000310509F0A5CF892F99276EC086E69CE0B3
:106CB0009F938F932F930E94341084E078CF80911C
:106CC000F203882309F451CF8091D30380FF4DCF85
:106CD0008091D503833009F048CF88EE94E00E947C
:106CE000F23A282F8823B1F583E39CE09F938F939A
:106CF0002F930E94341088EE94E00E94F33884E0D1
:106D000056CF84E08093E1048EE09CE09F938F93C4
:106D10001F920E9434100F900F900F909091E104F9
:106D200024CF84E08093E1048091E2049091E30415
:106D30009F938F938FEE9BE09F938F932F930E944F
:106D400034108AE090E00E9449139093E504809308
:106D5000E40487CF8091E6049091E7040E945213E7
:106D6000882309F400CF80E29EE40E9449139093A7
:106D7000E7048093E6048091E9049091EA040E947C
:106D80001A249091E104F1CEDF91CF910895CF9331
:106D9000DF93EC01892BD1F48091EB04833009F46B
:106DA0004AC01092EB04D093ED04C093EC0482EF40
:106DB00094E00E94C53BCE010E9449139093EF04DA
:106DC0008093EE048091EB0499270BC18091EE042F
:106DD0009091EF040E945213882329F49091EB04C0
:106DE000892F9927FEC0CE010E9449139093EF048A
:106DF0008093EE0480919E03823011F19091EB0418
:106E0000933071F782EF94E00E947A3B282F882319
:106E100009F479C08CEF9CE09F938F931F920E949E
:106E2000341082E08093EB040F900F900F90982F16
:106E3000892F9927D6C082EF94E00E947A3BB1CF88
:106E40009091EB04292F33272230310509F44CC0EF
:106E5000233031050CF04DC02115310509F444C033
:106E60002130310531F01092EB0490E0892F992701
:106E7000B8C00E9424359093ED048093EC040097F1
:106E800021F00E94FF318823A1F78091EC049091BA
:106E9000ED04009709F462C062EF74E00E94D63BF3
:106EA000282F882309F46AC080E29EE40E944913D7
:106EB0009093F1048093F00483E08093EB0480913D
:106EC000EC049091ED049F938F9381E89CE09F9355
:106ED0008F931F920E9434100F900F900F900F907D
:106EE0000F909091EB047CCF81E08093EB04982F7E
:106EF0009FCF2330310581F02430310509F0B3CF25
:106F0000892F99276EC081E19DE09F938F932F93E6
:106F10000E94341084E086CF8091F203882309F424
:106F20005FCF8091D30380FF5BCF8091D503833007
:106F300009F056CF82EF94E00E94753E282F8823F7
:106F4000B1F58EED9CE09F938F932F930E943410A8
:106F500082EF94E00E947A3B84E064CF84E08093E7
:106F6000EB0489EB9CE09F938F931F920E94341057
:106F70000F900F900F909091EB0432CF84E08093AC
:106F8000EB048091EC049091ED049F938F938AE938
:106F90009CE09F938F932F930E9434108AE090E09F
:106FA0000E9449139093EF048093EE0495CF809153
:106FB000F0049091F1040E945213882309F40ECF3B
:106FC00080E29EE40E9449139093F1048093F004C0
:106FD0008091F3049091F4040E941A249091EB04A0
:106FE000FFCEDF91CF9108950F931F9305E212E03A
:106FF00084EF91E09093260280932502B80180E00F
:107000000E94A63480E090E00E948C350E5F1F4FF6
:1070100088EE93E09093280280932702B80181E0E4
:107020000E94A63480E090E00E94C7361F910F9125
:1070300008951A9908958091F5049091F6040E949C
:1070400052138823B9F38AE090E00E944913909389
:10705000F6048093F5048091F704843041F0809128
:107060002502909126020E948C358093F70484308B
:1070700041F080912702909128020E94C7368093A8
:10708000F7048430B9F60E945A23882369F00E94DD
:10709000F4371092F7048AE090E00E94491390932D
:1070A000F6048093F504089588E893E10E9449135B
:1070B0009093F6048093F5040895FC0110821282E7
:1070C000118281E090E00895DF92EF92FF920F939A
:1070D0001F93CF93DF93EC017B01DD2461157105D4
:1070E00009F1CB010E945D3861E6CE010E94642D5A
:1070F000F70192838183892B99F081E0D82ED08289
:1071000005E21EE0C5EFD0E0F8010F5F1F4F84914C
:10711000F701618172810E94E12F2197D7FFF4CF9F
:107120006D2D7727CB01DF91CF911F910F91FF90AC
:10713000EF90DF900895EF92FF920F931F93CF93FC
:10714000DF937C0120E0FC0180818330B9F48181F0
:107150009281892B99F082E080830CE21DE0C0E2ED
:10716000D0E0F8010F5F1F4F8491F70161817281B8
:107170000E94E12F2197D7FFF4CF21E0822F99279A
:10718000DF91CF911F910F91FF90EF900895EF92B3
:10719000FF920F931F93CF93DF937C0120E0FC01BC
:1071A00080818230B9F481819281892B99F081E0CC
:1071B000808307EB1DE0CDE0D0E0F8010F5F1F4FAB
:1071C0008491F701618172810E94E12F2197D7FF9D
:1071D000F4CF21E0822F9927DF91CF911F910F915A
:1071E000FF90EF900895EF92FF920F931F93CF932C
:1071F000DF937C01009709F43DC0F701808188236B
:1072000079F099278230910589F1833091055CF4FA
:10721000019779F0F7011082F7018081882389F7BF
:1072200081E090E027C00397A9F7C7010E949B382F
:10723000E4CFF70181819281892B61F30FE01EE099
:10724000C4E1D0E0F8010F5F1F4F8491F701618125
:1072500072810E94E12F2197D7FFF4CFF70181813E
:1072600092810E94A524F7011082D6CFC7010E9407
:10727000C738C3CFDF91CF911F910F91FF90EF904F
:107280000895DF92EF92FF920F931F93CF93DF93B6
:107290007C01DD24FC0120812130B9F481819281BF
:1072A000892B99F082E08083D22E06EC1DE0C7E4A2
:1072B000D0E0F8010F5F1F4F8491F7016181728167
:1072C0000E94E12F2197D7FFF4CF8D2D9927DF91D1
:1072D000CF911F910F91FF90EF90DF900895EF9263
:1072E000FF920F931F93CF93DF937C0120E0FC016B
:1072F00080818230B9F481819281892B99F083E079
:1073000080830EE41DE0C7E6D0E0F8010F5F1F4F59
:107310008491F701618172810E94E12F2197D7FF4B
:10732000F4CF21E0822F9927DF91CF911F910F9108
:10733000FF90EF9008955F926F927F928F929F924D
:10734000AF92BF92CF92DF92EF92FF920F931F9373
:10735000CF93DF93CDB7DEB7E2970FB6F894DEBFD9
:107360000FBECDBF8C0120E0009709F425C18091AC
:10737000D203882319F4822F99271EC1F801808136
:107380008330C9F781819281892BA9F3C090C6030C
:10739000D090C703E090C803F090C903F7FCEAC09F
:1073A0003BE2532EC701B60120E836E948E950E038
:1073B0000E94E242490137FDFAC0C701B60120E848
:1073C00036E948E950E00E94E242DC01CB01BC0111
:1073D000CD0120E137E240E050E00E94E242590155
:1073E00037FDE0C0C701B60120E836E948E950E0C2
:1073F0000E94E242DC01CB01BC01CD0120E137E279
:1074000040E050E00E94E242DC01CB01BC01CD0132
:107410002AE030E040E050E00E94E242DA01C90197
:1074200097FDBCC03F932F93BF92AF929F928F92D4
:10743000852D99279F938F938BE692E09F938F934F
:107440003E010894611C711C7F926F920E94413F23
:10745000F80161817281C3010E948E31C090CA031C
:10746000D090CB03E090CC03F090CD038DB79EB7C6
:107470000C960FB6F8949EBF0FBE8DBFF7FC8BC065
:107480009BE2592EC701B60120E836E948E950E0F1
:107490000E94E242490137FD79C0C701B60120E8E8
:1074A00036E948E950E00E94E242DC01CB01BC0130
:1074B000CD0120E137E240E050E00E94E242590174
:1074C00037FD5FC0C701B60120E836E948E950E062
:1074D0000E94E242DC01CB01BC01CD0120E137E298
:1074E00040E050E00E94E242DC01CB01BC01CD0152
:1074F0002AE030E040E050E00E94E242DA01C901B7
:1075000097FD3BC03F932F93BF92AF929F928F9274
:10751000852D99279F938F938CE792E09F938F936C
:107520007F926F920E94413FF80161817281C30195
:107530000E948E311F921F921F921F928BE290E049
:107540009F938F938BE892E09F938F937F926F929C
:107550000E94413FF80161817281C3010E948E3116
:1075600021E08DB79EB746960FB6F8949EBF0FBE2A
:107570008DBF01CF4DE2542E15CF309521953F4F51
:10758000C1CFB094A194B108B3949CCF909481944E
:107590009108939482CF2DE2522E74CF309521958D
:1075A0003F4F40CFB094A194B108B3941BCF9094B7
:1075B00081949108939401CFE2960FB6F894DEBFC0
:1075C0000FBECDBFDF91CF911F910F91FF90EF9034
:1075D000DF90CF90BF90AF909F908F907F906F90F3
:1075E0005F900895CF93DF93EC0180E007C002978E
:1075F00021F5CE010E946F39813001F528812330B9
:10760000B1F0822F99278130910569F08230910580
:1076100074F7892B91F4BE0185E992E00E946438E9
:10762000813061F30BC0CE010E944139E5CF233098
:1076300029F4CE010E949B3901C080E09927DF9197
:10764000CF910895EF92FF920F931F93CF93DF9303
:107650007C0120E0FC0180818330B9F4818192813A
:10766000892B99F082E080830CE11FE0CAE0D0E032
:10767000F8010F5F1F4F8491F701618172810E94B1
:10768000E12F2197D7FFF4CF21E0822F9927DF91B7
:10769000CF911F910F91FF90EF900895EF92FF927D
:1076A0000F931F93CF93DF93EC0188818230C9F44D
:1076B00089819A81892BA9F081E0888383E3E82E70
:1076C0008FE0F82E07E010E0F7010894E11CF11CB0
:1076D000849169817A810E94E12F0150104017FF47
:1076E000F3CF80E090E0DF91CF911F910F91FF9059
:1076F000EF900895EF92FF920F931F93CF93DF9334
:10770000EC01009709F43AC08881882369F0992731
:107710008230910579F1833091054CF4019769F03D
:1077200018828881882399F781E090E027C0039729
:10773000B9F7CE010E94223BE7CF89819A81892B3C
:1077400079F39BE5E92E9FE0F92E07E010E0F701C1
:107750000894E11CF11C849169817A810E94E12FD7
:107760000150104017FFF3CF89819A810E94A52410
:107770001882D7CFCE010E944E3BC6CFDF91CF916A
:107780001F910F91FF90EF900895CF93DF93EC013D
:107790008881882319F0CE010E947A3B18821A82D0
:1077A000198281E090E0DF91CF910895DF92EF920E
:1077B000FF920F931F93CF93DF93EC017B01DD24A6
:1077C0006115710509F1CB010E94C53B61E6CE014F
:1077D0000E94642DF70192838183892B99F021E027
:1077E000D22ED08204E61FE0CAECD0E0F8010F5F91
:1077F0001F4F8491F701618172810E94E12F2197CF
:10780000D7FFF4CF6D2D7727CB01DF91CF911F915B
:107810000F91FF90EF90DF900895DF92EF92FF922B
:107820000F931F93CF93DF937C01DD24FC01208114
:107830002130B9F481819281892B99F082E0808393
:10784000D22E0CE31FE0CDE1D0E0F8010F5F1F4F17
:107850008491F701618172810E94E12F2197D7FF06
:10786000F4CF8D2D9927DF91CF911F910F91FF902C
:10787000EF90DF900895EF92FF920F931F93CF93B5
:10788000DF937C0120E0FC0180818230B9F48181AA
:107890009281892B99F083E0808308E21FE0C9E0A0
:1078A000D0E0F8010F5F1F4F8491F7016181728171
:1078B0000E94E12F2197D7FFF4CF21E0822F992753
:1078C000DF91CF911F910F91FF90EF9008955F92FC
:1078D0006F927F928F929F92AF92BF92CF92DF92E0
:1078E000EF92FF920F931F93CF93DF93CDB7DEB745
:1078F000C456D0400FB6F894DEBF0FBECDBF8C018A
:1079000020E0009709F4DAC18091D203882319F4AA
:10791000822F9927D3C1D8018C918330C9F7F80100
:1079200081819281892BA1F3C090CA03D090CB03AF
:10793000E090CC03F090CD03F7FC9EC15BE2552EA6
:10794000C701B60120E836E948E950E00E94E2426A
:10795000390137FDAEC1C701B60120E836E948E973
:1079600050E00E94E242DC01CB01BC01CD0120E1EC
:1079700037E240E050E00E94E242590137FD94C1F5
:10798000C701B60120E836E948E950E00E94E2422A
:10799000DC01CB01BC01CD0120E137E240E050E049
:1079A0000E94E242DC01CB01BC01CD012AE030E0C3
:1079B00040E050E00E94E242DA01C90197FD70C147
:1079C0003F932F93BF92AF927F926F92852D99270D
:1079D0009F938F9381EA92E09F938F934E01089437
:1079E000811C911C9F928F920E94413FF8016181FE
:1079F0007281C4010E948E31C090C603D090C7032B
:107A0000E090C803F090C9038DB79EB70C960FB6EF
:107A1000F8949EBF0FBE8DBFF7FC3FC13BE2532ED3
:107A2000C701B60120E836E948E950E00E94E24289
:107A3000390137FD2DC1C701B60120E836E948E913
:107A400050E00E94E242DC01CB01BC01CD0120E10B
:107A500037E240E050E00E94E242590137FD13C195
:107A6000C701B60120E836E948E950E00E94E24249
:107A7000DC01CB01BC01CD0120E137E240E050E068
:107A80000E94E242DC01CB01BC01CD012AE030E0E2
:107A900040E050E00E94E242DA01C90197FDEFC0E8
:107AA0003F932F93BF92AF927F926F92852D99272C
:107AB0009F938F938DEB92E09F938F939F928F92E2
:107AC0000E94413FF80161817281C4010E948E31A0
:107AD0008091A20699279F938F938091A106992761
:107AE0009F938F938091A00699279F938F93809166
:107AF0009F0699279F938F9380919E0699279F9326
:107B00008F9380919C0690919D069F938F9385ED16
:107B100092E09F938F939F928F920E94413FF80132
:107B200061817281C4010E948E318091D4039927B2
:107B30009F938F9383E093E09F938F939F928F9275
:107B40000E94413F8DB79EB782960FB6F8949EBFB4
:107B50000FBE8DBFF80161817281C4010E948E3118
:107B60008FE0E3E1F3E0D40101900D928A95E1F713
:107B7000F80161817281C4010E948E318091EA0313
:107B80009091EB03A091EC03B091ED03BC01CD010A
:107B900020EA36E841E050E00E94E2423F932F9312
:107BA00082E293E09F938F939F928F920E94413F36
:107BB000F80161817281C4010E948E318091E603D7
:107BC0009091E7039F938F938AE393E09F938F9322
:107BD0009F928F920E94413FF80161817281C4019E
:107BE0000E948E312091000130910101C9016AE0AB
:107BF00070E00E94AD42562EC9016AE070E00E941A
:107C0000AD4299279F938F93852D99279F938F93AB
:107C10008AE593E09F938F939F928F920E94413FBA
:107C2000F80161817281C4010E948E3180E1E7E731
:107C3000F3E0D40101900D928A95E1F7F80161819A
:107C40007281C4010E948E318BE0E7E8F3E0D40139
:107C500001900D928A95E1F7F80161817281C4016A
:107C60000E948E3121E08DB79EB744960FB6F894EE
:107C70009EBF0FBE8DBF4CCE6DE2562E61CE3095AD
:107C800021953F4F0DCFB094A194B108B394E8CEA5
:107C90007094619471087394CECE4DE2542EC0CE90
:107CA000309521953F4F8CCEB094A194B108B394F8
:107CB00067CE70946194710873944DCECC59DF4FA8
:107CC0000FB6F894DEBF0FBECDBFDF91CF911F91ED
:107CD0000F91FF90EF90DF90CF90BF90AF909F906B
:107CE0008F907F906F905F900895CF93DF93EC011A
:107CF00080E007C0029721F5CE010E943B3C813015
:107D000001F528812330B1F0822F99278130910528
:107D100069F08230910574F7892B91F4BE0182E9F4
:107D200093E00E94D63B813061F30BC0CE010E94EC
:107D30000D3CE5CF233029F4CE010E94673C01C001
:107D400080E09927DF91CF910895FC01882799273A
:107D5000E89421912223F1F02032D9F32930C9F39C
:107D60002A30B9F32C30A9F32D3099F3263789F353
:107D70002B3219F02D3221F468942191222351F0F5
:107D8000203344F02A3334F420530E94393F820FC9
:107D9000911DF3CF8115910521F01EF480959095EA
:107DA00001960895FB01DC0140FF05C002C005906B
:107DB0000D9205900D9242505040C8F70895FC0175
:107DC0004150504030F001900616D1F73197CF0165
:107DD0000895882799270895FB01DC0140FF05C01D
:107DE00002C001900D9201900D9242505040C8F790
:107DF0000895FB01DC014150504030F08D9101901D
:107E0000801919F40020B9F7881B990B0895009781
:107E100031F4DA018D919C91009709F40EC0DC01D8
:107E2000FB013D912191222319F03217C9F3FACFBA
:107E3000332331F4DA011D921C9288279927089583
:107E40001197AF93BF93FB013D912191321771F4CC
:107E5000332321F488279927119702C01E92119687
:107E6000FA01A193B0839F918F910895222369F71E
:107E7000EACF7AE0979F902D879F802D910D112456
:107E800008950F931F93CF93DF93CDB7DEB72E974F
:107E90000FB6F894DEBF0FBECDBF0D891E892F89A6
:107EA000388D86E08C831A8309838FEF9FE79E834A
:107EB0008D83AE01475E5F4FB901CE0101960E94EE
:107EC000713FEF81F885E00FF11F10822E960FB6FB
:107ED000F894DEBF0FBECDBFDF91CF911F910F9100
:107EE00008952F923F924F925F926F927F928F925E
:107EF0009F92AF92BF92CF92DF92EF92FF920F9339
:107F00001F93CF93DF93CDB7DEB762970FB6F89488
:107F1000DEBF0FBECDBFEE24FF2487011C017E878C
:107F20006D872A01CC24DD24FC01D782C68283819F
:107F300081FD68C28FEF9FEF78C28D859E85019687
:107F40009E878D87C0FE4BC28F8580538A30D0F4C8
:107F50009F85903339F4662029F4C3FC03C0E0E028
:107F6000F1E08DC08AE0689E602C1124FF856F0EC1
:107F700020ED620E67FE02C05FE7652EC3FC42C2C1
:107F8000762C40C2C3FE04C0662011F441E0642E8A
:107F9000EF858E2F992787FD9095883691058CF572
:107FA000853691050CF06EC08335910509F493C0B8
:107FB00084359105CCF48B32910509F449C08C329B
:107FC00091054CF48032910509F446C08332910545
:107FD00009F44AC0FEC18D32910509F440C08E32C9
:107FE000910509F444C0F5C18336910509F450C0E8
:107FF000843691050CF08AC08835910509F4BCC01F
:10800000E8C18037910509F4B1C08137910584F446
:108010008C36910591F18D3691052CF489369105B8
:1080200009F474C0D6C18F36910509F49CC0D1C142
:108030008537910509F4A2C08637910524F483376A
:10804000910571F1C6C18837910509F495C0C1C188
:1080500080E190E0C82AD92AE0E2F0E010C080E890
:1080600090E0C82AD92ACEC1E0E4F0E008C088E058
:1080700090E0C82AD92A6624C5C1E4E0F0E0CE2AFF
:10808000DF2AC0C13FE3E32E7A94F3E6FF873CC1C9
:10809000F20182E090E0480E591EE0807A9434C1EB
:1080A000F20182E090E0480E591EA081B1817D016D
:1080B000C3FE09C0862D992787FD9095BC01CD018F
:1080C0000E9442421FC0FD0101900020E9F7319754
:1080D000EA1BE88B18C0F20182E090E0480E591EBE
:1080E0000190F081E02D7F01C3FE09C0862D992704
:1080F00087FD9095BC01CF010E94374203C0CF019C
:108100000E942E42888B9889791AFEC0C2FE0AC04E
:10811000F20184E090E0480E591E208131814281B5
:1081200053810CC0F20182E090E0480E591E80811C
:1081300091819C01442737FD4095542F79018A0194
:1081400057FF0CC0E2E0F0E0CE2ADF2A1095009540
:10815000F094E094E11CF11C011D111D8FEB9FEFC9
:10816000C822D92227C098E0988B08C0E0E4F0E04C
:10817000CE2ADF2AF8E7FF8720E1288BC2FE0AC05B
:10818000F20184E090E0480E591E20813181428145
:1081900053810AC0F20182E090E0480E591E8081AE
:1081A00091819C014427552779018A01EFECFFEF6B
:1081B000CE22DF22CE0101969A8B898B9889892E57
:1081C0009924AA24BB24C801B701A50194010E94E7
:1081D000C042DC01CB01E989FA8980838A3024F02E
:1081E000FF858F0F815201C0805DE989FA898193F3
:1081F000FA8BE98BC801B701A50194010E94C04226
:1082000079018A012115310541055105E1F6E98819
:1082100081E090E08C0F9D1FE81AC6018273907078
:10822000892B09F07A94C6FE0DC0872D992787FD0A
:108230009095E889E03121F42EEF722E780E02C07D
:10824000782E7A94C3FE0FC0262D332727FD309554
:108250008E2D9927821793072CF087EF9FEFC82266
:10826000D92201C06E18C3FE02C0761801C07E1864
:10827000C60180789170892B51F4872D7A94181655
:1082800034F4B10180E290E00E944D42F6CFC1FE8D
:1082900004C0B1018DE290E00BC0C4FE04C0B10186
:1082A0008BE290E005C0C5FE05C0B10180E290E020
:1082B0000E944D42C6FE10C0B10180E390E00E94D2
:1082C0004D429889903141F4B101EF858E2F992765
:1082D00087FD90950E944D42D0FE0AC0872D7A946A
:1082E000181634F4B10180E390E00E944D42F6CFBD
:1082F000C3FE0AC0862D6A94181634F4B10180E3D7
:1083000090E00E944D42F6CF90E8B92EBC2051F487
:10831000872D7A94181634F4B10180E290E00E941F
:108320004D42F6CFFF85F33641F48E2DB1019927EA
:1083300087FD90950E944D4240C02F852337B1F4B0
:1083400088898150888B8F3FC1F1F7018081089423
:10835000E11CF11CB101992787FD90950E944D42C7
:1083600098899150988B9F3F81F727C0EF85E3351F
:1083700079F4F889F150F88BFF3FF9F0F701849117
:10838000B10199270E944D420894E11CF11CF1CFE4
:108390006E010894C11CD11C89899A898C159D0590
:1083A00061F0E989FA898291FA8BE98BB101992709
:1083B00087FD90950E944D42EFCFBB2069F0872D3D
:1083C0007A9418164CF4B10180E290E00E944D427C
:1083D000F6CFB1010E944D42CC24DD2413C09F850D
:1083E000953241F481E0C82ED12C6624762CEAE047
:1083F000E88B08C0B101FF858F2F992787FD9095E5
:108400000E944D42F101838183FF04C0ED85FE850A
:10841000F49103C0ED85FE85F081FF872F8522232F
:1084200009F08BCDF1018681978162960FB6F894A1
:10843000DEBF0FBECDBFDF91CF911F910F91FF9097
:10844000EF90DF90CF90BF90AF909F908F907F90F4
:108450006F905F904F903F902F900895FC01059092
:108460000020E9F7809590958E0F9F1F0895FC01DD
:108470000590615070400110D8F7809590958E0F4F
:108480009F1F0895FC016150704001900110D8F7C2
:10849000809590958E0F9F1F08950F931F93CF93F4
:1084A000DF938C01EB018B81992781FF1CC082FF38
:1084B0000DC02E813F818C819D812817390764F47E
:1084C000E881F9810193F983E88306C0E885F9859D
:1084D000802F0995892B39F48E819F8101969F8386
:1084E0008E83C80102C08FEF9FEFDF91CF911F9164
:1084F0000F910895629FD001739FF001829FE00D5C
:10850000F11D649FE00DF11D929FF00D839FF00D12
:10851000749FF00D659FF00D9927729FB00DE11DBE
:10852000F91F639FB00DE11DF91FBD01CF0111249B
:108530000895AA1BBB1B51E107C0AA1FBB1FA617AA
:10854000B70710F0A61BB70B881F991F5A95A9F7FC
:1085500080959095BC01CD01089597FB092E0726C3
:108560000AD077FD04D0E5DF06D000201AF470951C
:1085700061957F4F0895F6F7909581959F4F0895E7
:10858000A1E21A2EAA1BBB1BFD010DC0AA1FBB1F17
:10859000EE1FFF1FA217B307E407F50720F0A21B89
:1085A000B30BE40BF50B661F771F881F991F1A94F6
:1085B00069F760957095809590959B01AC01BD0120
:1085C000CF01089597FB092E05260ED057FD04D044
:1085D000D7DF0AD0001C38F450954095309521958E
:1085E0003F4F4F4F5F4F0895F6F7909580957095E8
:0A85F00061957F4F8F4F9F4F089554
:1085FA0078006401FFFFFF48656C6C6F20576F724B
:10860A006C64000000000000000000000000000090
:10861A000000000000000000000000000000000050
:10862A000000000000000000000000000000000040
:10863A000000000000000000000000000000000030
:10864A000000000000000003000000001F000000FE
:10865A003B0000005A00000078000000970000006C
:10866A00B5000000D4000000F30000001101000072
:10867A00300100004E0100006D0100000000000002
:10868A001F0000003C0000005B00000079000000B1
:10869A0098000000B6000000D5000000F4000000B9
:1086AA0012010000310100004F0100006E010000BC
:1086BA0001004B4D4C4C6F6767696E672020202084
:1086CA0020200001F401F401000060EA014750583B
:1086DA004C6F6767696E672020202020200001E820
:1086EA0003E803000060EA20202020202020202028
:1086FA0020202020202020000073657474696E6792
:10870A00732E696E69003D002573203D2025640D96
:10871A000A000D0A00F401E8034C4F472F253034B4
:10872A006925303269253032692F4B4D4C2F47501D
:10873A0053253035692E4B4D4C004C4F472F253071
:10874A00346925303269253032692F4750582F470E
:10875A005053253035692E475058000D0A25632598
:10876A00642E252E3364252E33642C00256325645C
:10877A002E252E3364252E33642C00256325642E82
:10878A00252E33640064656661756C742E6B6D6C9E
:10879A00003C74726B7074206C61743D22256325F1
:1087AA00642E252E3364252E33642220006C6F6ECE
:1087BA003D22256325642E252E3364252E3364221B
:1087CA00203E0D0A003C74696D653E253034642DE7
:1087DA00253032642D2530326454253032643A25EE
:1087EA003032643A253032645A3C2F74696D653EE2
:1087FA000D0A003C7361743E25643C2F7361743E1C
:10880A000D0A003C657874656E73696F6E733E0D70
:10881A000A003C436F757273653E253033643C2F02
:10882A00436F757273653E0D0A003C47726F756E31
:10883A006453706565643E25643C2F47726F756E9C
:10884A006453706565643E0D0A003C566F6C746132
:10885A0067653E25642E253031643C2F566F6C7453
:10886A006167653E0D0A003C2F657874656E736911
:10887A006F6E733E0D0A003C2F74726B70743E0D5E
:0E888A000A0064656661756C742E6770780074
:00000001FF
